:020000040000FA
:3D000000FFFF627F2100FFFFFFFFFFFFFFFFFFFFFFFFFFFFFFFFFFFFFFFFFFFFFFFFFFFFFFFFFFFFFFFFFFFFFFFFFFFFFFFFFFFFFFFFFFFFFFFFFFFFFFFFFFFFFFFA
:3D003D00601886611896611886611896611886611886651886611896611886010000000018866118866118866118866118866518866118866518866118866180F2EA
:3D007A0040100441100E41100441100E41100441108443100441100E411004010000000010044110044110044110044110844310044110844310044110044180CD5E
:3D00B700000000000000000000000000000000000000000000000000000000000000000000000000000000000000000000000000000000000000000000000080E7A5
:3D00F400000000000000000000000000000000000000000000000000000000000000000000000000000000000000000000000000000000000000000000000080E768
:3D013100000000000008000000000008000000000000020000000008000000000000000000000000000000000000000000000200000000000200000000000000ED86
:3D016E0000000000000A00000000000A00000000009000000000000A000000000000000000000000000000000000000000800200000000800200000000000080DE44
:3D01AB00000000000000000000000000000000000000000000000000000000000000000000000000000000000000000000000000000000000000000000000080E7B0
:3D01E800000000000000000000000000000000000000000000000000000000000000000000000000000000000000000000000000000000000000000000000090F654
:3D022500000000000000000000000000000000000000000000000000000000000000000000000000000000000000000000000000000000000000000000000080E735
:3D026200000000000000000000000000000000000000000000000000000000000000000000000000000000000000000000000000000000000000000000000080E7F8
:3D029F00000000000000000000000000000000000000000000000000000000000000000000000000000000000000000000000000000000000000000000000080E7BB
:3D02DC00000000000000000000000000000000000000000000000000000000000000000000000000000000000000000000000000000000000000000000000080E77E
:3D031900000000000000000000000000000000000000000000000000000000000000000000000000000000000000000000000000000000000000000000000080E740
:3D035600000000000000000000000000000000000000000000000000000000000000000000000000000000000000000000000000000000000000000000000048AB77
:3D039300000000000000000000000000000000000000000000000000000000000000000000000000000000000000000000000000000000000000000000000080E7C6
:3D03D000000000000000000000000000000000000000000000000000000000000000000000000000000000000000000000000000000000000000000000000080E789
:3D040D00000000000000000000000000000000000000000000000000000000000000000000000000000000000000000000000000000000000000000000000080E74B
:3D044A00000000000000000000000000000000000000000000000000000000000000000000000000000000000000000000000000000000000000000000000080E70E
:3D048700000000000000000000000000000000000000000000000000000000000000000000000000000000000000000000000000000000000000000000000080E7D1
:3D04C4000000000000000000000000000000000000000000000000000000000000000000000000000000000000000000000000000000000000000000000000A0C596
:3D050100000000000000000000000000000000000000000000000000000000000000000000000000000000000000000000000000000000000000000000000080E756
:3D053E00000000000000000000000000000000000000000000000000000000000000000000000000000000000000000000000000000000000000000000000080E719
:3D057B00000000000000000000000000000000000000000000000000000000000000000000000000000000000000000000000000000000000000000000000080E7DC
:3D05B800000000000000000000000000000000000000000000000000000000000000000000000000000000000000000000000000000000000000000000000080E79F
:3D05F500000000000000000000000000000000000000000000000000000000000000000000000000000000000000000000000000000000000000000000000080E762
:3D063200000000000000000000000000000000000000000000000000000000000000000000000000000000000000000000000000000000000000000000000080E724
:3D066F00000000000000000000000000000000000000000000000000000000000000000000000000000000000000000000000000000000000000000000000058BA3C
:3D06AC00000000000000000000000000000000000000000000000000000000000000000000000000000000000000000000000000000000000000000000000080E7AA
:3D06E900000000000000000000000000000004000000100000000000000000000000000000000000000000000800000000002000000000000000000000000000B5E3
:3D072600000000000000000000000000000000000000000000000000000000000000000000000000000000000000000000000000000000000000000000000080E72F
:3D076300000000000000000000000000000000000000000000000000000000000000000000000000000000000000000000000000000000000000000000000080E7F2
:3D07A000000000000000000000000000000000000000000000000000000000000000000000000000000000000000000000000000000000000000000000000080E7B5
:3D07DD0000000000000000000000000000000400000010000000000000000000000000000000000000000000080000000000A000000000000000000000000000BD66
:3D081A00000110000110000110000110000110000110000110000110000110000000000040000440000440000440000440000440000440000440000440000480E73D
:3D085700000000000000000000000000000000000000000000000000000000000000000000000000000000000000000000000000000000000000000000000080E7FD
:3D089400800118800118800118800118800118800118800118800118800118000000000060000660000660000660000660000660000660000660000660000608EF39
:3D08D100820008800008800008800008800008800008800008800008800008000000000020000220000220000220000220000220000220000220000220000208EDF9
:3D090E00020000000000000000000000000000000000080000000000000000000000000000000000000000000000000000000000000000000000000000000090FC16
:3D094B000200000000000000000000000000000000060000000000000000000000000000000000000000000000000000000000000000000000000000000000088DD2
:3D098800020000000000000000000000000000000000000000000000000000000000000000000000000000000000000000000000000000000000000000000008ED3B
:3D09C500000000000000000000000000000000000004000000000000000000000000000000000000000000000000000000000000000000000000000000000008AF3A
:3D0A0200000000000000000000000000000000000018000000000000000000000000000000000000000000000000000000000000000000000000000000000000FEA1
:3D0A3F00000000000000000000000000000000000018000000000000000000000000000000000000000000000000000000000000000000000000000000000000FE64
:3D0A7C00000000000000000000000000000000000018000000000000000000000000000000000000000000000000000000000000000000000000000000000000FE27
:3D0AB900000000000000000000000000000000000018000000000000000000000000000000000000000000000000000000000000000000000000000000000088F66A
:3D0AF600020000000000000000000000000000000000000000000000000000000000000000000000000000000000000000000000000000000000000000000008EDCC
:3D0B3300020000000000000000000000000000000000000000000000000000000000000000000000000000000000000000000000000000000000000000000090F4FF
:3D0B7000020000000000000000000000000000000000000000000000000000000000000000000000000000000000000000000000000000000000000000000008ED51
:3D0BAD00020000000000000000000000000000000000000000000000000000000000000000000000000000000000000000000000000000000000000000000008ED14
:3D0BEA00000000000000000000000000000000000000000000000000000000000000000000000000000000000000000000000000000000000000000000000008EFD7
:3D0C2700000000000000000000000000000000000000000000000000000000000000000000000000000000000000000000000000000000000000000000000080E729
:3D0C6400000000000000000000000000000000000000000000000000000000000000000000000000000000000000000000000000000000000000000000000008EF5C
:3D0CA100020000000000000000000000000000000000000000000000000000000000000000000000000000000000000000000000000000000000000000000008ED1F
:3D0CDE00020000000000000000000000000000000000000000000000000000000000000000000000000000000000000000000000000000000000000000000090F453
:3D0D1B00020000000000000000000000000000000000000000000000000000000000000000000000000000804100000098400000000000000000000000000088A9CF
:3D0D5800020000000000000000000000000000000000000000000000000000000000000000000000000000000000000000000000000000000000000000000008ED67
:3D0D9500000000000000000000000000000000000000000000000000000000000000000000000000000000000100000010000000000000000000000000000008EF19
:3D0DD200000000000000000000000000000000000000000000000000000000000000000000000000000000000600000060000000000000000000000000000080E717
:3D0E0F00000000000000000000000000000000000000000000000000000000000000000000000000000000000600000060000000000000000000000000000080E7D9
:3D0E4C00000000000000000000000000000000000000000000000000000000000000000000000000000000000600000060000000000000000000000000000080E79C
:3D0E8900000000000000000000000000000000000000000000000000000000000000000000000000000000000600000060000000000000000000000000000008EFCF
:3D0EC600020000000000000000000000000000000000000000000000000000000000000000000000000000000000000000000000000000000000000000000008EDF8
:3D0F0300020000000000000000000000000026080000000000000000000000000000000000000000000000000000000000000000000000000000000000000090BE33
:3D0F4000020000000000000000000000000000000000000000000000000000000000000000000000000000000000000000000000000000000000000000000008ED7D
:3D0F7D00020000000000000000000000000004000000000000000000000000000000000000000000000000000000000000000000000000000000000000000008AD7C
:3D0FBA00000000000000000000000000000018000000000000000000000000000000000000000000000000000000000000000000000000000000000000000088F664
:3D0FF700000000000000000000000000000018000000000000000000000000000000000000000000000000000000000000000000000000000000000000000000FEA7
:3D103400000000000000000000000000000018000000000000000000000000000000000000000000000000000000000000000000000000000000000000000088F6E9
:3D107100020000000000000000000000000018000000000000000000000000000000000000000000000000000000000000000000000000000000000000000088F4AC
:3D10AE00020000000000000000000000000000000000000000000000000000000000000000000000000000000000000000000000000000000000000000000090F47F
:3D10EB00020000000000000000000000000000000000000000000000000000000000000000000000000000000000000000000000000000000000000000000008EDD1
:3D112800020000000000000000000000000000000000000000000000000000000000000000000000000000000000000000000000000000000000000000000008ED93
:3D116500000000000000000000000000000000000000000000000000000000000000000000000000000000000000000000000000000000000000000000000008EF56
:3D11A200000000000000000000000000000000000000000000000000000000000000000000000000000000000000000000000000000000000000000000000080E7A9
:3D11DF00000000000000000000000000000000000000000000000000000000000000000000000000000000000000000000000000000000000000000000000080E76C
:3D121C00000000000000000000000000000000000000000000000000000000000000000000000000000000000000000000000000000000000000000000000080E72E
:3D125900000000000000000000000000000000000000000000000000000000000000000000000000000000000000000000000000000000000000000000000008EF61
:3D129600020000000000000000000000000000000000000000000000000000000000000000000000000000000000040000000000000000000000000000000008E924
:3D12D300020000000000000000000000000000000000000000000000000000000000000000000000000000000098000000000000000000000000000000000090EDC7
:3D131000020000000000000000000000000000000000000000000000000000000000000000000000000000000000000000000000000000000000000000000008EDA9
:3D134D00020000000000000000000000000000000000000000000000000000000000000000000000000000000010000000000000000000000000000000000008FC4D
:3D138A000000000000000000000000000000000000000000000000000000000000000000000000000000000000600000000000000000000000000000000000088935
:3D13C7000000000000000000000000000000000000000000000000000000000000000000000000000000000000600000000000000000000000000000000000808188
:3D14040000000000000000000000000000000000000000000000000000000000000000000000000000000000006000000000000000000000000000000000000889BA
:3D1441000200000000000000000000000000000000000000000000000000000000000000000000000000000000600000000000000000000000000000000000088B79
:3D147E00020000000000000000000000000000000001000000000000000000000000000000000000000000000000000000000000000000000000000000000090E4BA
:3D14BB00020000000000000000000000000000600200000000000000000000000000000000000000000000000000000000000000000000000000000000000008AFD9
:3D14F800020000000000000000000000000000000000000000000000000000000000000000000000000000000000000000000000000000000000000000000008EDC0
:3D153500000000000000000000000000000000400000000000000000000000000000000000000000000000000000000000000000000000000000000000000008AF82
:3D157200000000000000000000000000000000800100000000000000000000000000000000000000000000000000000000000000000000000000000000000000FEBD
:3D15AF00000000000000000000000000000000800100000000000000000000000000000000000000000000000000000000000000000000000000000000000000FE80
:3D15EC00000000000000000000000000000000800100000000000000000000000000000000000000000000000000000000000000000000000000000000000000FE43
:3D162900000000000000000000000000000000800100000000000000000000000000000000000000000000000000000000000000000000000000000000000000FE05
:3D166600020000000000000000000000000001000000000000000000000000000000000000000000000080000000000000000000000000000000000000000088FD3F
:3D16A300020000000000000000000000600000000000000000000000000000000000000000000000000018000000800102000000000000000000000000000008AD58
:3D16E000020000000000000000000000000000000000000000000000000000000000000000000000000000000000000000000000000000000000000000000008EDD6
:3D171D00020000000000000000000000400000000000000000000000000000000000000000000000000010000000000100000000000000000000000000000008AD87
:3D175A00000000000000000000000000800100000000000000000000000000000000000000000000000060000000000600000000000000000000000000000000FE6D
:3D1797001E0000000000000000000000800100000000000000000000000000000000000000000000000060000000000600000000000000000000000000000000E030
:3D17D4001E0000000000000000000000800100000000000000000000000000000000000000000000000060000000000600000000000000000000000000000088E863
:3D181100000000000000000000000000800100000000000000000000000000000000000000000000000060000000000600000000000000000000000000000000FEB5
:3D184E00000110000110000110000110000110000110000110000110000110000000000040000440000440000440000440000440000440000440000440000480E7F9
:3D188B00000000000000000000000000000000000000000000000000000000000000000000000000000000000000000000000000000000000000000000000080E7B9
:3D18C800800118800118800118800118800118800118800118800118800118000000000060000660000660000660000660000660000660000660000660000680E785
:3D190500800008800008800008800008800008800008800008800008800008000000000020000220000220000220000220000220000220000220000220000280E744
:3D1942000000000000000000000000000000500000000300000000000000000000000000000000000000000000000000030000000000000000000000000000808111
:3D197F00000000000000000000000000000000000000000000000000000000000000000000000000000000000000000000000000000000000000000000000080E7C4
:3D19BC00000000000000000000000000000000000000000000000000000000000000000000000000000000000000000000000000000000000000000000000080E787
:3D19F900000000000000000000000000000000000000000000000000000000000000000000000000000020000000000200000000000000000000000000000080E728
:3D1A3600000000000000000000000000000040000000010000000000000000000000000000000000000000000000000002000000000000000000000000000080822E
:3D1A7300000000000000000000000000000000000000000000000000000000000000000000000000000000000000000000000000000000000000000000000080E7CF
:3D1AB0000000000000000000000000000000000000000000000000000000000000000000000000000000000000000000000000000000000000000000000000C0A396
:3D1AED00000000000000000000000000000000000000000000000000000000000000000000000000000000000000008000000000000000000000000000000080EFCD
:3D1B2A00000000000000000000000000000000008000000000000000000000000000000000000000000000000020000000000000000000000000000000000080CD91
:3D1B6700000000000000000000000000000000040000000000000000000000000000000000000000000010000400000000000000000000000000000000000080B6F3
:3D1BA4000000000000000000000000000000010000000200000000000000000000000000000000000000000000000000000000000000000000000000000000D0A091
:3D1BE100000000000000000000000000000000000000000000000000000000000000000000000000000000000000000000000000000000000000000000000080E760
:3D1C1E00000000000000000000000000000000000000000000000000000000000000000000000000000000000000000000000000000000000000000000000080E722
:3D1C5B00000000000000000000000000000000000000000000000000000000000000000000000000000000000000000000200000000000000000000000000080C7E5
:3D1C9800000000000000000000000000000000000000000000000000000000000000000000000000000000000000000000000000000000000000000000000080E7A8
:3D1CD500000000000000000000000000000000000000000000000000000000000000000000000000000000000000000000000000000000000000000000000080E76B
:3D1D1200000000000000000000000000000000000000000000000000000000000000000000000000000000000000000000000000000000000000000000000080E72D
:3D1D4F00000000000000000000000000000000000000000000000000000000000000000000000000000000000000000000000000000000000000000000000080E7F0
:3D1D8C00000000000000000000000000000000000000000000000000000000000000000000000000000000000000000000000000000000000000000000000080E7B3
:3D1DC900000000000000000000000000000000000000000000000000000000000000000000000000000000000000000000000000000000000000000000000080E776
:3D1E06000000000000000000000000000000000000000000000000000000000000000000000000000000000000000000000000000000000000000000000000A0C53A
:3D1E4300000000000000000000000000000000000000000000000000000000000000000000000000000000000000000000000000000000000000000000000080E7FB
:3D1E8000000000000000000000000000000000000000000000000000000000000000000000000000000000000000000000000000000000000000000000000080E7BE
:3D1EBD00000000000000000000000000000000000000000000000000000000000000000000000000000000000000000000000000000000000000000000000080E781
:3D1EFA00000000000000000000000000000000000000000000000000000000000000000000000000000000000000000000000000000000000000000000000080E744
:3D1F3700000000000000000000000000000000000000000000000000000000000000000000000000000000000000000000000000000000000000000000000080E706
:3D1F7400000000000000000000000000000000000000000000000000000000000000000000000000000000000000000000000000000000000000000000000080E7C9
:3D1FB100000000000000000000000000000000000000000000000000000000000000000000000000000000000000000000000000000000000000000000000080E78C
:3D1FEE000000000000000000000000000000000000000000000000000000000000000000000000000000000000000000000000000000000000000000000000A0C551
:3D202B00000000000000000000000000000000000000000000000000000000000000000000000000000000000000000000000000000000000000000000000080E711
:3D206800000000000000000000000000000000000000000000000000000000000000000000000000000000000000000000000000000000000000000000000080E7D4
:3D20A500000000000000000000000000000000000000000000000000000000000000000000000000000000000000000000000000000000000000000000000080E797
:3D20E200000000000000000000000000000000000000000000000000000000000000000000000000000000000000000000000000000000000000000000000090F63B
:3D211F00000000000000000000000000000000000000000000000000000000000000000000000000000000000000000000000000000000000000000000000080E71C
:3D215C00000000000000000000000000000000000000000000000000000000000000000000000000000000000000000000000000000000000000000000000080E7DF
:3D219900000000000000000000000000000000000000000000000000000000000000000000000000000000000000000000000000000000000000000000000080E7A2
:3D21D600000000000000000000000000000000000000000000000000000000000000000000000000000000000000000000000000000000000000000000000080E765
:3D221300000000000000000000000000000000000000000000000000000000000000000000000000000000000000000000000000000000000000000000000080E727
:3D225000000000000000000000000000000000000000000000000000000000000000000000000000000000000000000000000000000000000000000000000080E7EA
:3D228D00000000000000000000000000000000000000000000000000000000000000000000000000000000000000000000000000000000000000000000000080E7AD
:3D22CA000000000000000000000000000000000000000000000000000000000000000000000000000000000000000000000000000000000000000000000000C0A374
:3D230700000000000000000000000000000000000000000000000000000000000000000000000000000000000000000000000000000000000000000000000080E732
:3D234400000000000000000000000000000000000000000000000000000000000000000000000000000000000000000000000000000000000000000000000080E7F5
:3D238100000000000000000000000000000000000000000000000000000000000000000000000000000000000000000000000000000000000000000000000080E7B8
:3D23BE00000000000000000000000000000000000000000000000000000000000000000000000000000000000000000000000000000000000000000000000080E77B
:3D23FB00000000000000000000000000000000000000000000000000000000000000000000000000000000000000000000000000000000000000000000000008EFAE
:3D243800000000000000000000000000000000000000000000000000000000000000000000000000000000000000000000000000000000000000000000000080E700
:3D2475000000000000000000000000000000000000000000000000000000000000000000000000000000000000000000000000000000000000000000000000B0D4A6
:3D24B200000000000000000000000000000000000000000000000000000000000000000000000000000000000000000000000000000000000000000000000080E786
:3D24EF0000000000000000000000000000000000000000004000000000000000000000000000000000000000000000000000000A00200000000000000000000089BD
:3D252C00000000000000000000000000000000000000000000000000000000000000000000000000000000000000000000000000000000000000000000000080E70B
:3D256900000000000000000000000000000000000000000000000000000000000000000000000000000000000000000000000000000000000000000000000080E7CE
:3D25A600000000000000000000000000000000000000000000000000000000000000000000000000000000000000000000000000000000000000000000000080E791
:3D25E30000000000000000000000000000000000000000004000000000000000000000000000000000000000000000000000000A00200000000000000000000089C8
:3D262000000110000110000110000110000110000110000110000110000110000000000040000440000440000440000440000440000440000440000440000480E719
:3D265D00000000000000000000000000000000000000000000000000000000000000000000000000000000000000000000000000000000000000000000000080E7D9
:3D269A00800118800118800118800118800118800118800118800118800118000000000060000660000660000660000660000660000660000660000660000608EF15
:3D26D700820008800008800008800008800008800008800008800008800008000000000020000220000220000220000220000220000220000220000220000208EDD5
:3D271400020000000000000000000000000000000000000000000000000000000000000000000000000000000000000000000800000000000000000000000010F47A
:3D275100020000000000000000000000000000000000000000000000000000000000000000000000000000000000000000800100000000000000000000000088F44C
:3D278E00020000000000000000000000000000000000000000000000000000000000000000000000000000000000000000000000000000000000000000000008ED17
:3D27CB00000000000000000000000000000000000000000000000000000000000000000000000000000000000000000000000100000000000000000000000008FECA
:3D280800000000000000000000000000000000000000000000000000000000000000000000000000000000000000000000000600000000000000000000000080818C
:3D284500000000000000000000000000000000000000000000000000000000000000000000000000000000000000000000000600000000000000000000000080814F
:3D2882000000000000000000000000000000000000000000000000000000000000000000000000000000000000000000000006000000000000000000000000808112
:3D28BF000000000000000000000000000000000000000000000000000000000000000000000000000000000000000000000006000000000000000000000000088945
:3D28FC00020000000000000000000000000000000000000000000000000000000000000000000000000000000000000000000000000004000000000000000008ADE4
:3D293900020000000000000000000000000000000000000000000000000000000000000000000000000000000000000000000000800900000000000000000090ED59
:3D297600020000000000000000000000000000000000000000000000000000000000000000000000000000000000000000000000000000000000000000000008ED2D
:3D29B300020000000000000000000000000000000000000000000000000000000000000000000000000000000000000000000000000100000000000000000008FCE0
:3D29F0000000000000000000000000000000000000000000000000000000000000000000000000000000000000000000000000000006000000000000000000088913
:3D2A2D000000000000000000000000000000000000000000000000000000000000000000000000000000000000000000000000000006000000000000000000808165
:3D2A6A000000000000000000000000000000000000000000000000000000000000000000000000000000000000000000000000000006000000000000000000088998
:3D2AA7000200000000000000000000000000000000000000000000000000000000000000000000000000000000000000000000000006000000000000000000088B57
:3D2AE400020000000000000000000000000000000000000000000000000000000000000000000000000000000000000000000000000000000000000000000090F42F
:3D2B2100020000000000000000000000000000000000000026100000000000000000000000000000000000000000000000000000000000000000000000000008BF78
:3D2B5E00020000000000000000000000000000000000000000000000000000000000000000000000000000000000000000000000000000000000000000000008ED43
:3D2B9B00000000000000000000000000000000000000000004000000000000000000000000000000000000000000000000000000000000000000000000000008AF42
:3D2BD800000000000000000000000000000000000000000018000000000000000000000000000000000000000000000000000000000000000000000000000000FEAA
:3D2C1500000000000000000000000000000000000000000018000000000000000000000000000000000000000000000000000000000000000000000000000000FE6C
:3D2C5200000000000000000000000000000000000000000018000000000000000000000000000000000000000000000000000000000000000000000000000000FE2F
:3D2C8F00000000000000000000000000000000000000000018000000000000000000000000000000000000000000000000000000000000000000000000000088F672
:3D2CCC00020000000000000000000000000000000000000000000000000000000000000000000000000000000000000000000000200000000000000000000008CDD4
:3D2D0900020000000000000000000000000000000000000000000000000000000000000000000000000000000000000000000018000000000000000000000010ED76
:3D2D4600020000000000000000000000000000000000000000000000000000000000000000000000000000000000000000000000000000000000000000000008ED59
:3D2D8300020000000000000000000000000000000000000000000000000000000000000000000000000000000000000000000010000000000000000000000008FCFD
:3D2DC00000000000000000000000000000000000000000000000000000000000000000000000000000000000000000000000006000000000000000000000000889E5
:3D2DFD000000000000000000000000000000000000000000000000000000000000000000000000000000000000000000000000600000000000000000000000808138
:3D2E3A00000000000000000000000000000000000000000000000000000000000000000000000000000000000000000000000060000000000000000000000008896A
:3D2E77000200000000000000000000000000000000000000000000000000000000000000000000000000000000000000000000600000000000000000000000088B29
:3D2EB400020000000000000000000000000000000000000000000000000000000000000000000000000000000000000000000000000000000000000000000090F45B
:3D2EF100020000000000000000000000000000000000000000000000000000000000000000000000000000000000000000000000000000000000000000000008EDAD
:3D2F2E00020000000000000000000000000000000000000000000000000000000000000000000000000000000000000000000000000000000000000000000008ED6F
:3D2F6B00000000000000000000000000000000000000000000000000000000000000000000000000000000000000000000000000000000000000000000000008EF32
:3D2FA800000000000000000000000000000000000000000000000000000000000000000000000000000000000000000000000000000000000000000000000080E785
:3D2FE500000000000000000000000000000000000000000000000000000000000000000000000000000000000000000000000000000000000000000000000080E748
:3D302200000000000000000000000000000000000000000000000000000000000000000000000000000000000000000000000000000000000000000000000080E70A
:3D305F00000000000000000000000000000000000000000000000000000000000000000000000000000000000000000000000000000000000000000000000008EF3D
:3D309C00020000000000000000000000000000000000000000000000000000000000000000000000000000000000000000000000000000400000000000000008AD00
:3D30D900020000000000000000000000000000000000000000000000000000000000000000000000000000000000000000000000000018000000000000000010EDA3
:3D311600020000000000000000000000000000000000000000000000000000000000000000000000000000000000000000000000000000000000000000000008ED85
:3D315300020000000000000000000000000000000000000000000000000000000000000000000000000000000000000000000000000010000000000000000008FC29
:3D3190000000000000000000000000000000000000000000000000000000000000000000000000000000000000000000000000000000600000000000000000088911
:3D31CD000000000000000000000000000000000000000000000000000000000000000000000000000000000000000000000000000000600000000000000000808164
:3D320A000000000000000000000000000000000000000000000000000000000000000000000000000000000000000000000000000000600000000000000000088996
:3D3247000200000000000000000000000000000000000000000000000000000000000000000000000000000000000000000000000000600000000000000000088B55
:3D328400020000000000000000000000000000000000001000000000000000000000000000000000000000000000000000000000000000000000000000000090F576
:3D32C100020000000000000000000000000000000000600200000000000000000000000000000000000000000000000000000000000000000000000000000008AFB5
:3D32FE00020000000000000000000000000000000000000000000000000000000000000000000000000000000000000000000000000000000000000000000008ED9C
:3D333B00000000000000000000000000000000000000400000000000000000000000000000000000000000000000000000000000000000000000000000000008AF5E
:3D337800000000000000000000000000000000000000800100000000000000000000000000000000000000000000000000000000000000000000000000000000FE99
:3D33B500000000000000000000000000000000000000800100000000000000000000000000000000000000000000000000000000000000000000000000000000FE5C
:3D33F200000000000000000000000000000000000000800100000000000000000000000000000000000000000000000000000000000000000000000000000000FE1F
:3D342F00000000000000000000000000000000000000800100000000000000000000000000000000000000000000000000000000000000000000000000000000FEE1
:3D346C00020000000000000000000000000000000000000000000000000000000000000000000000000000000000000000000000000000000000000000000008ED2C
:3D34A900020000000000000000000000000000000000000000608006010000000000000000000000000000000000000000000000000000800902000000000008DD8D
:3D34E600020000000000000000000000000000000000000000000000000000000000000000000000000000000000000000000000000000000000000000000008EDB2
:3D352300020000000000000000000000000000000000000000400004000000000000000000000000000000000000000000000000000000000100000000000008FC20
:3D356000000000000000000000000000000000000000000000800118000000000000000000000000000000000000000000000000000000000600000000000080818E
:3D359D001E00000000000000000000000000000000000000008001180000000000000000000000000000000000000000000000000000000006000000000000809F15
:3D35DA001E00000000000000000000000000000000000000008001180000000000000000000000000000000000000000000000000000000006000000000000089758
:3D36170000000000000000000000000000000000000000000080011800000000000000000000000000000000000000000000000000000000060000000000008081D6
:3D365400000110000110000110000110000110000110000110000110000110000000000040000440000440000440000440000440000440000440000440000480E7D5
:3D369100000000000000000000000000000000000000000000000000000000000000000000000000000000000000000000000000000000000000000000000080E795
:3D36CE00800118800118800118800118800118800118800118800118800118000000000060000660000660000660000660000660000660000660000660000680E761
:3D370B00800008800008800008800008800008800008800008800008800008000000000020000220000220000220000220000220000220000220000220000280E720
:3D37480000000000000000000000000000000000000000000003005000000000000000000000000000000000000000000000000000000000000300000000008081ED
:3D378500000000000000000000000000000000000000000000000000000000000000000000000000000000000000000000000000000000000000000000000080E7A0
:3D37C200000000000000000000000000000000000000000000000000000000000000000000000000000000000000000000000000000000000000000000000080E763
:3D37FF00000000000000000000000000000000000000000000000008000000000000000000000000000000000000000000000000000000000200000000000000CDB6
:3D383C00000000000000000000000000000000000000000000010040000000000000000000000000000000000000000000000000000000000002000000000080820A
:3D387900000000000000000000000000000000000000000000000000000000000000000000000000000000000000000000000000000000000000000000000080E7AB
:3D38B6000000000000000000000000000000000000000000000000000000000000000000000000000000000000000000000000000000000000000000000000E08174
:3D38F3000000000000000000000000000000000000000000000020000000000000000000000000000000000000000000000000000000000000000000000000C0A117
:3D393000000000000000000000000000000000000000800000000000000000000000000000000000000000000000000000000000000002000000000000000000CF09
:3D396D00000000000000000000000000000000000000000000000010000000000000000000000000000000000000000000000100000000000001000000000080F794
:3D39AA00000000000000000000000000000000000000000000000000000000000000000000000000000000000000000000000000080000400000000000000080AF69
:3D39E700000000000000000000000000000000000000000000000000000000000000000000000000000000000000000000000000000000000000000000000080E73C
:3D3A2400000000000000000000000000000000000000000000000000000000000000000000000000000000000000000000000000000000000000000000000080E7FE
:3D3A61000000000000000000000000000000000000000000000800000000000000000000000000000000000000000000000000000000000000000000000000B0DC94
:3D3A9E00000000000000000000000000000000000000000000000000000000000000000000000000000000000000000000000000000000000000000000000080E784
:3D3ADB00000000000000000000000000000000000000000000000000000000000000000000000000000000000000000000000000000000000000000000000080E747
:3D3B1800000000000000000000000000000000000000000000000000000000000000000000000000000000000000000000000000000000000000000000000080E709
:3D3B5500000000000000000000000000000000000000000000000000000000000000000000000000000000000000000000000000000000000000000000000080E7CC
:3D3B9200000000000000000000000000000000000000000000000000000000000000000000000000000000000000000000000000000000000000000000000080E78F
:3D3BCF00000000000000000000000000000000000000000000000000000000000000000000000000000000000000000000000000000000000000000000000080E752
:3D3C0C00000000000000000000000000000000000000000000000000000000000000000000000000000000000000000000000000000000000000000000000080E714
:3D3C4900000000000000000000000000000000000000000000000000000000000000000000000000000000000000000000000000000000000000000000000080E7D7
:3D3C8600000000000000000000000000000000000000000000000000000000000000000000000000000000000000000000000000000000000000000000000080E79A
:3D3CC300000000000000000000000000000000000000000000000000000000000000000000000000000000000000000000000000000000000000000000000080E75D
:3D3D0000000000000000000000000000000000000000000000000000000000000000000000000000000000000000000000000000000000000000000000000080E71F
:3D3D3D00000000000000000000000000000000000000000000000000000000000000000000000000000000000000000000000000000000000000000000000080E7E2
:3D3D7A00000000000000000000000000000000000000000000000000000000000000000000000000000000000000000000000000000000000000000000000080E7A5
:3D3DB7000000000000000000000000000000000000000000000000000000000000000000000000000000000000000000000000000000000000000000000000B0D44B
:3D3DF4000000000000000000000000000000000000000000000000000000000000000000000000000000000000000000000000000000000000000000000000C0A32F
:3D3E3100000000000000000000000000000000000000000000000000000000000000000000000000000000000000000000000000000000000000000000000080E7ED
:3D3E6E00000000000000000000000000000000000000000000000000000000000000000000000000000000000000000000000000000000000000000000000080E7B0
:3D3EAB00000000000000000000000000000000000000000000000000000000000000000000000000000000000000000000000000000000000000000000000080E773
:3D3EE800000000000000000000000000000000000000000000000000000000000000000000000000000000000000000000000000000000000000000000000080E736
:3D3F2500000000000000000000000000000000000000000000000000000000000000000000000000000000000000000000000000000000000000000000000080E7F8
:3D3F6200000000000000000000000000000000000000000000000000000000000000000000000000000000000000000000000000000000000000000000000080E7BB
:3D3F9F00000000000000000000000000000000000000000000000000000000000000000000000000000000000000000000000000000000000000000000000080E77E
:3D3FDC00000000000000000000000000000000000000000000000000000000000000000000000000000000000000000000000000000000000000000000000080E741
:3D401900000000000000000000000000000000000000000000000000000000000000000000000000000000000000000000000000000000000000000000000080E703
:3D405600000000000000000000000000000000000000000000000000000000000000000000000000000000000000000000000000000000000000000000000080E7C6
:3D409300000000000000000000000000000000000000000000000000000000000000000000000000000000000000000000000000000000000000000000000080E789
:3D40D000000000000000000000000000000000000000000000000000000000000000000000000000000000000000000000000000000000000000000000000008EFBC
:3D410D00000000000000000000000000000000000000000000000000000000000000000000000000000000000000000000000000000000000000000000000080E70E
:3D414A00000000000000000000000000000000000000000000000000000000000000000000000000000000000000000000000000000000000000000000000080E7D1
:3D418700000000000000000000000000000000000000000000000000000000000000000000000000000000000000000000000000000000000000000000000080E794
:3D41C400000000000000000000000000000000000000000000000000000000000000000000000000000000000000000000000000000000000000000000000080E757
:3D420100000000000000000000000000000000000000000000000000000000000000000000000000000000000000000000000000000000000000000000000080E719
:3D423E00000000000000000000000000000000000000000000000000000000000000000000000000000000000000000000000000000000000000000000000080E7DC
:3D427B00000000000000000000000000000000000000000000000000000000000000000000000000000000000000000000000000000000000080000000000050B284
:3D42B800000000000000000000000000000000000000000000000000000000000000000000000000000000000000000000000000000000000000000000000080E762
:3D42F5000000000000000000000000000000000000000000000000000000400000000000000000020000000000000000000000000000000000000000080020008999
:3D433200000000000000000000000000000000000000000000000000000000000000000000000000000000000000000000000000000000000000000000000080E7E7
:3D436F00000000000000000000000000000000000000000000000000000000000000000000000000000000000000000000000000000000000000000000000080E7AA
:3D43AC00000000000000000000000000000000000000000000000000000000000000000000000000000000000000000000000000000000000000000000000080E76D
:3D43E9000000000000000000000000000000000000000000000000000000400000000000000000030000000000000000000000000000000000000000080020009993
:3D442600000110000110000110000110000110000110000110000110000110000000000040000440000440000440000440000440000440000440000440000480E7F5
:3D446300000000000000000000000000000000000000000000000000000000000000000000000000000000000000000000000000000000000000000000000080E7B5
:3D44A000800118800118800118800118800118800118800118800118800118000000000060000660000660000660000660000660000660000660000660000608EFF1
:3D44DD00820008800008800008800008800008800008800008800008800008000000000020000220000220000220000220000220000220000220000220000208EDB1
:3D451A00020000000000000000000000000000000000000000000000000000000000000000000000000000000000000000000000000000000000000000000090F4DE
:3D455700020000000000000000000000000000000000000000000000000000000000000000000000000000000000000000000000000000000000000000000008ED30
:3D459400020000000000000000000000000000000000000000000000000000000000000000000000000000000000000000000000000000000000000000000008EDF3
:3D45D100000000000000000000000000000000000000000000000000000000000000000000000000000000000000000000000000000000000000000000000008EFB6
:3D460E00000000000000000000000000000000000000000000000000000000000000000000000000000000000000000000000000000000000000000000000080E708
:3D464B00000000000000000000000000000000000000000000000000000000000000000000000000000000000000000000000000000000000000000000000080E7CB
:3D468800000000000000000000000000000000000000000000000000000000000000000000000000000000000000000000000000000000000000000000000080E78E
:3D46C500000000000000000000000000000000000000000000000000000000000000000000000000000000000000000000000000000000000000000000000008EFC1
:3D47020002000000000000000000000000000000000000000000000000000000000000000000000000000000000000000000000000000000000000000000000CADBF
:3D473F00020000000000000000000000000000000000000000000000000000000000000098400000000000000000000000000000000000000000000000800990B496
:3D477C00020000000000000000000000000000000000000000000000000000000000000000000000000000000000000000000000000000000000000000000008ED09
:3D47B900020000000000000000000000000000000000000000000000000000000000000010000000000000000000000000000000000000000000000000000108EDBB
:3D47F600000000000000000000000000000000000000000000000000000000000000000060000000000000000000000000000000000000000000000000000608EF29
:3D483300000000000000000000000000000000000000000000000000000000000000000060000000000000000000000000000000000000000000000000000680E77B
:3D487000000000000000000000000000000000000000000000000000000000000000000060000000000000000000000000000000000000000000000000000608EFAE
:3D48AD00020000000000000000000000000000000000000000000000000000000000000060000000000000000000000000000000000000000000000000000608ED71
:3D48EA00020000000000000000000000000000000000000000000000000000080000000000000000000000000000000000000000000000000000000000000090FCFB
:3D4927000200000000000000000000000000000000000000000000000000060000000000000000000000000000000000000000000000000000000000000000088DB6
:3D496400020000000000000000000000000000000000000000000000000000000000000000000000000000000000000000000000000000000000000000000008ED1F
:3D49A100000000000000000000000000000000000000000000000000000004000000000000000000000000000000000000000000000000000000000000000008AF1E
:3D49DE00000000000000000000000000000000000000000000000000000018000000000000000000000000000000000000000000000000000000000000000000FE86
:3D4A1B00000000000000000000000000000000000000000000000000000018000000000000000000000000000000000000000000000000000000000000000000FE48
:3D4A5800000000000000000000000000000000000000000000000000000018000000000000000000000000000000000000000000000000000000000000000000FE0B
:3D4A9500000000000000000000000000000000000000000000000000000018000000000000000000000000000000000000000000000000000000000000000088F64E
:3D4AD200020000000000000000000000000000000000000000000000000000000000000000000000000000000000000000000000000000000000000000400008ADB0
:3D4B0F00020000000000000000000000000000000000000000000000000000000000000000000000000000000000000000000000000000000000000018000010ED52
:3D4B4C00020000000000000000000000000000000000000000000000000000000000000000000000000000000000000000000000000000000000000000000008ED35
:3D4B8900020000000000000000000000000000000000000000000000000000000000000000000000000000000000000000000000000000000000000010000008FCD9
:3D4BC60000000000000000000000000000000000000000000000000000000000000000000000000000000000000000000000000000000000000000006000000889C1
:3D4C03000000000000000000000000000000000000000000000000000000000000000000000000000000000000000000000000000000000000000000600000808113
:3D4C40000000000000000000000000000000000000000000000000000000000000000000000000000000000000000000000000000000000000000000600000088946
:3D4C7D000200000000000000000000000000000000000000000000000000000000000000000000000000000000000000000000000000000000000000600000088B05
:3D4CBA00020000000000000000000000000000000000000000000000000000000000000000000000000000000000000000000000000000000000000000000090F437
:3D4CF700020000000000000000000000000000000000000000000000000000000000000000000000000000000000000000000000000000000000804100000088F045
:3D4D3400020000000000000000000000000000000000000000000000000000000000000000000000000000000000000000000000000000000000000000000008ED4B
:3D4D7100000000000000000000000000000000000000000000000000000000000000000000000000000000000000000000000000000000000000000100000008FEFE
:3D4DAE0000000000000000000000000000000000000000000000000000000000000000000000000000000000000000000000000000000000000000060000008081C1
:3D4DEB000000000000000000000000000000000000000000000000000000000000000000000000000000000000000000000000000000000000000006000000808184
:3D4E28000000000000000000000000000000000000000000000000000000000000000000000000000000000000000000000000000000000000000006000000808146
:3D4E65000000000000000000000000000000000000000000000000000000000000000000000000000000000000000000000000000000000000000006000000088979
:3D4EA200020000000000000000000000000000000000000000000000000000000000000000000000000000000000000000000000000000000000000000000008EDDC
:3D4EDF00020000000000000000000000000000000000000000000000000000000000000000000000000000000000000000000000000000000000000000000090F410
:3D4F1C00020000000000000000000000000000000000000000000000000000000000000000000000000000000000000000000000000000000000000000000008ED61
:3D4F5900020000000000000000000000000000000000000000000000000000000000000000000000000000000000000000000000000000000000000000000008ED24
:3D4F9600000000000000000000000000000000000000000000000000000000000000000000000000000000000000000000000000000000000000000000000008EFE7
:3D4FD300000000000000000000000000000000000000000000000000000000000000000000000000000000000000000000000000000000000000000000000080E73A
:3D501000000000000000000000000000000000000000000000000000000000000000000000000000000000000000000000000000000000000000000000000008EF6C
:3D504D00020000000000000000000000000000000000000000000000000000000000000000000000000000000000000000000000000000000000000000000008ED2F
:3D508A00020000000000000000000000000000000000000000000000001000000000000000000000000000000000000000000000000000000000000000000090F552
:3D50C700020000000000000000000000000000000000000000000000600200000000000000000000000000000000000000000000000000000000000000000008AF91
:3D510400020000000000000000000000000000000000000000000000000000000000000000000000000000000000000000000000000000000000000000000008ED77
:3D514100000000000000000000000000000000000000000000000000400000000000000000000000000000000000000000000000000000000000000000000008AF3A
:3D517E00000000000000000000000000000000000000000000000000800100000000000000000000000000000000000000000000000000000000000000000000FE75
:3D51BB00000000000000000000000000000000000000000000000000800100000000000000000000000000000000000000000000000000000000000000000000FE38
:3D51F800000000000000000000000000000000000000000000000000800100000000000000000000000000000000000000000000000000000000000000000000FEFB
:3D523500000000000000000000000000000000000000000000000000800100000000000000000000000000000000000000000000000000000000000000000088F63D
:3D527200020200000000000000000000000000000000000000000000000000000000000000000000000000000000000000000000000000000000000000000008CF24
:3D52AF00620006080000000000000000000000000000000000000000000000000000000000000000000000000000000000000000000000000018080000000010ED35
:3D52EC00020000000000000000000000000000000000000000000000000000000000000000000000000000000000000000000000000000000000000000000008ED8E
:3D532900420004000000000000000000000000000000000000000000000000000000000000000000000000000000000000000000000000000010000000000008FCED
:3D5366008001180000000000000000000000000000000000000000000000000000000000000000000000000000000000000000000000000000600000000000088980
:3D53A3009E01180000000000000000000000000000000000000000000000000000000000000000000000000000000000000000000000000000600000000000809F97
:3D53E0009E01180000000000000000000000000000000000000000000000000000000000000000000000000000000000000000000000000000600000000000809F5A
:3D541D008001180000000000000000000000000000000000000000000000000000000000000000000000000000000000000000000000000000600000000000808158
:3D545A00000110000110000110000110000110000110000110000110000110000000000040000440000440000440000440000440000440000440000440000480E7B1
:3D549700000000000000000000000000000000000000000000000000000000000000000000000000000000000000000000000000000000000000000000000080E771
:3D54D400800118800118800118800118800118800118800118800118800118000000000060000660000660000660000660000660000660000660000660000680E73D
:3D551100800008800008800008800008800008800008800008800008800008000000000020000220000220000220000220000220000220000220000220000280E7FC
:3D554E00000050000000000000000000000000000000000000000000000000030000000000000000000000000000000000000000000000000008000002000000992A
:3D558B00000000000000000000000000000000000000000000000000000000000000000000000000000000000000000000000000000000000000000000000080E77C
:3D55C800000000000000000000000000000000000000000000000000000000000000000000000000000000000000000000000000000000000000000000000080E73F
:3D560500000008000000000000000000000000000000000000000000000000000000000000000000000000000000000000000000000000000000000000000000EF71
:3D5642000000400000000000000000000000000000000000000000000000000100000000000000000000000000000000000000000000000000080000020000008A56
:3D567F00000000000000000000000000000000000000000000000000000000000000000000000000000000000000000000000000000000000000000000000080E787
:3D56BC00000000000000000000000000000000000000000000000000000000000000000000000000000000000000000000000000000000000000000000000028CDBC
:3D56F900000000020000000000000000000000000000000000000000000000000000000000000000000000000000000000000000000000000000000000000080E50D
:3D573600000000000000000000000000000000000000000000000000800000000000000000000000000000000000000000000000000000000000000000000012DEC6
:3D577300400000000000000000000000000000000000000000000000000000000000000000000000000000000000000000000000000000000000000400000080E352
:3D57B000000000000000000000000000000000000000000000000000000000020000000000000000000000000000000000000000000000000000000000400080A555
:3D57ED00000000000000000000000000000000000000000000000000000000000000000000000000000000000000000000000000000000000000000000000080E718
:3D582A00000000000000000000000000000000000000000000000000000000000000000000000000000000000000000000000000000000000000000000000080E7DA
:3D586700000000000000000000000000000000000000000000000000000000000000000000200000000000000000000000000000000000000000000000000080C79D
:3D58A400000000000000000000000000000000000000000000000000000000000000000000000000000000000000000000000000000000000000000000000080E760
:3D58E100000000000000000000000000000000000000000000000000000000000000000000000000000000000000000000000000000000000000000000000008EF93
:3D591E000000000000000000000000000000000000000000000000000000000000000000000000000000000000000000000000000000000000000000000000A0C5E7
:3D595B00000000000000000000000000000000000000000000000000000000000000000000000000000000000000000000000000000000000000000000000080E7A8
:3D599800000000000000000000000000000000000000000000000000000000000000000000000000000000000000000000000000000000000000000000000080E76B
:3D59D5000000000000000000000000000000000000000000000000000000000000000000000000000000000000000000000000000000000000000000000000C0A332
:3D5A1200000000000000000000000000000000000000000000000000000000000000000000000000000000000000000000000000000000000000000000000080E7F0
:3D5A4F00000000000000000000000000000000000000000000000000000000000000000000000000000000000000000000000000000000000000000000000080E7B3
:3D5A8C00000000000000000000000000000000000000000000000000000000000000000000000000000000000000000000000000000000000000000000000080E776
:3D5AC900000000000000000000000000000000000000000000000000000000000000000000000000000000000000000000000000000000000000000000000080E739
:3D5B0600000000000000000000000000000000000000000000000000000000000000000000000000000000000000000000000000000000000000000000000080E7FB
:3D5B4300000000000000000000000000000000000000000000000000000000000000000000000000000000000000000000000000000000000000000000000080E7BE
:3D5B8000000000000000000000000000000000000000000000000000000000000000000000000000000000000000000000000000000000000000000000000080E781
:3D5BBD000000000000000000000000000000000000000000000000000000000000000000000000000000000000000000000000000000000000000000000000C0A348
:3D5BFA000000000000000000000000000000000000000000000000000000000000000000000000000000000000000000000000000000000000000000000000B0D4EA
:3D5C3700000000000000000000000000000000000000000000000000000000000000000000000000000000000000000000000000000000000000000000000080E7C9
:3D5C7400000000000000000000000000000000000000000000000000000000000000000000000000000000000000000000000000000000000000000000000080E78C
:3D5CB100000000000000000000000000000000000000000000000000000000000000000000000000000000000000000000000000000000000000000000000080E74F
:3D5CEE00000000000000000000000000000000000000000000000000000000000000000000000000000000000000000000000000000000000000000000000080E712
:3D5D2B00000000000000000000000000000000000000000000000000000000000000000000000000000000000000000000000000000000000000000000000008EF44
:3D5D6800000000000000000000000000000000000000000000000000000000000000000000000000000000000000000000000000000000000000000000000080E797
:3D5DA500000000000000000000000000000000000000000000000000000000000000000000000000000000000000000000000000000000000000000000000080E75A
:3D5DE200000000000000000000000000000000000000000000000000000000000000000000000000000000000000000000000000000000000000000000000080E71D
:3D5E1F00000000000000000000000000000000000000000000000000000000000000000000000000000000000000000000000000000000000000000000000080E7DF
:3D5E5C00000000000000000000000000000000000000000000000000000000000000000000000000000000000000000000000000000000000000000000000080E7A2
:3D5E9900000000000000000000000000000000000000000000000000000000000000000000000000000000000000000000000000000000000000000000000080E765
:3D5ED600000000000000000000000000000000000000000000000000000000000000000000000000000000000000000000000000000000000000000000000080E728
:3D5F1300000000000000000000000000000000000000000000000000000000000000000000000000000000000000000000000000000000000000000000000080E7EA
:3D5F5000000000000000000000000000000000000000000000000000000000000000000000000000000000000000000000000000000000000000000000000080E7AD
:3D5F8D00000000000000000000000000000000000000000000000000000000000000000000000000000000000000000000000000000000000000000000000080E770
:3D5FCA00000000000000000000000000000000000000000000000000000000000000000000000000000000000000000000000000000000000000000000000080E733
:3D600700000000000000000000000000000000000000000000000000000000000000000000000000000000000000000000000000000000000000000000000080E7F5
:3D604400000000000000000000000000000000000000000000000000000000000000000000000000000000000000000000000000000000000000000000000080E7B8
:3D608100000000000000000000000000000000000000000000000000000000000000000000000000000000000000000000000000000000000000000000000058BAD0
:3D60BE00000000000000000000000000000000000000000000000000000000000000000000000000000000000000000000000000000000000000000000000080E73E
:3D60FB00000000000000100000010000000000000000000000000000000000000000000000000008000000000800000000000000000000000000000000000080FEC9
:3D613800000000000000000000000000000000000000000000000000000000000000000000000000000000000000000000000000000000000000000000000080E7C3
:3D617500000000000000000000000000000000000000000000000000000000000000000000000000000000000000000000000000000000000000000000000080E786
:3D61B200000000000000000000000000000000000000000000000000000000000000000000000000000000000000000000000000000000000000000000000080E749
:3D61EF00000000000000140000010000000000000000000000000000000000000000000000000008000000000800000000000000000000000000000000000080FAD4
:3D622C00000110000110000110000110000110000110000110000110000110000000000040000440000440000440000440000440000440000440000440000480E7D1
:3D626900000000000000000000000000000000000000000000000000000000000000000000000000000000000000000000000000000000000000000000000080E791
:3D62A600800118800118800118800118800118800118800118800118800118000000000060000660000660000660000660000660000660000660000660000608EFCD
:3D62E300820008800008800008800008800008800008800008800008800008000000000020000220000220000220000220000220000220000220000220000208ED8D
:3D632000020000000000000000000000000000000000000000000000000000000000000000000000000000000000000000000000000000000000000000000090F4BA
:3D635D00020000000000000000000000000000000000000000000000000000000000000000000000000000000000000000000000000000000000000000000008ED0C
:3D639A00020000000000000000000000000000000000000000000000000000000000000000000000000000000000000000000000000000000000000000000008EDCF
:3D63D700000000000000000000000000000000000000000000000000000000000000000000000000000000000000000000000000000000000000000000000008EF92
:3D641400000000000000000000000000000000000000000000000000000000000000000000000000000000000000000000000000000000000000000000000080E7E4
:3D645100000000000000000000000000000000000000000000000000000000000000000000000000000000000000000000000000000000000000000000000080E7A7
:3D648E00000000000000000000000000000000000000000000000000000000000000000000000000000000000000000000000000000000000000000000000080E76A
:3D64CB00000000000000000000000000000000000000000000000000000000000000000000000000000000000000000000000000000000000000000000000008EF9D
:3D650800020000000001000000000000000000000000000000000000000000000000000000000000000000000000000000000000000000000000000000000008FD4E
:3D654500020000600200000006010000000000000000000000000000000000000000000000000000000000000000000000000000000000000000000000000090D747
:3D658200020000000000000000000000000000000000000000000000000000000000000000000000000000000000000000000000000000000000000000000008EDE5
:3D65BF00020000400000000004000000000000000000000000000000000000000000000000000000000000000000000000000000000000000000000000000008ED64
:3D65FC00000000800100000018000000000000000000000000000000000000000000000000000000000000000000000000000000000000000000000000000008EFD2
:3D663900000000800100000018000000000000000000000000000000000000000000000000000000000000000000000000000000000000000000000000000080E724
:3D667600000000800100000018000000000000000000000000000000000000000000000000000000000000000000000000000000000000000000000000000008EF57
:3D66B300020000800100000018000000000000000000000000000000000000000000000000000000000000000000000000000000000000000000000000000008ED1A
:3D66F000020000000000000000000000000000000000000000000000000000000000000000000000000000004000000000000000000000000000000000000090F0AB
:3D672D00020000000000000000000000000000000000000000000000000000000000000000000000000000800900000000000000000000000000000000000008F4A8
:3D676A00020000000000000000000000000000000000000000000000000000000000000000000000000000000000000000000000000000000000000000000008EDFB
:3D67A700000000000000000000000000000000000000000000000000000000000000000000000000000000000100000000000000000000000000000000000008FEAE
:3D67E4000000000000000000000000000000000000000000000000000000000000000000000000000000000006000000000000000000000000000000000000808171
:3D6821000000000000000000000000000000000000000000000000000000000000000000000000000000000006000000000000000000000000000000000000808133
:3D685E0000000000000000000000000000000000000000000000000000000000000000000000000000000000060000000000000000000000000000000000008081F6
:3D689B000000000000000000000000000000000000000000000000000000000000000000000000000000000006000000000000000000000000000000000000088929
:3D68D800020000000000000000000000000000000000000000000000000000000000000000000000000000000000000000000000000000000000000000000008ED8C
:3D691500020000000000000000000000000000000000000000000000000000000000000000000098400000000000000000000000000000000000000000000090AD2E
:3D695200020000000000000000000000000000000000000000000000000000000000000000000000000000000000000000000000000000000000000000000008ED11
:3D698F00020000000000000000000000000000000000000000000000000000000000000000000010000000000000000000000000000000000000000000000008FCB5
:3D69CC00000000000000000000000000000000000000000000000000000000000000000000000060000000000000000000000000000000000000000000000008899D
:3D6A090000000000000000000000000000000000000000000000000000000000000000000000006000000000000000000000000000000000000000000000008081EF
:3D6A46000000000000000000000000000000000000000000000000000000000000000000000000600000000000000000000000000000000000000000000000088922
:3D6A83000200000000000000000000000000000000000000000000000000000000000000000000600000000000000000000000000000000000000000000000088BE1
:3D6AC000020000000000080000000000000000000000000000000000000000000000000000000000000000000000000000000000000000000000000000000090FC03
:3D6AFD000200000000060000000000000000000000000000000000000000000000000000000000000000000000000000000000000000000000000000000000088DBF
:3D6B3A00020000000000000000000000000000000000000000000000000000000000000000000000000000000000000000000000000000000000000000000008ED27
:3D6B7700000000000004000000000000000000000000000000000000000000000000000000000000000000000000000000000000000000000000000000000008AF26
:3D6BB400000000000018000000000000000000000000000000000000000000000000000000000000000000000000000000000000000000000000000000000000FE8E
:3D6BF100000000000018000000000000000000000000000000000000000000000000000000000000000000000000000000000000000000000000000000000000FE51
:3D6C2E00000000000018000000000000000000000000000000000000000000000000000000000000000000000000000000000000000000000000000000000000FE13
:3D6C6B00000000000018000000000000000000000000000000000000000000000000000000000000000000000000000000000000000000000000000000000088F656
:3D6CA800020000000000000000000000000000000000000000000000000000000000000000000000000000000000000000000000000000000000000000000008EDB8
:3D6CE500020000000000000000000000000000000000000000000000000000000000000000000000800102000000000000000000000000000000000000000010CD10
:3D6D2200020000000000000000000000000000000000000000000000000000000000000000000000000000000000000000000000000000000000000000000008ED3D
:3D6D5F00020000000000000000000000000000000000000000000000000000000000000000000000000100000000000000000000000000000000000000000008FCF0
:3D6D9C000000000000000000000000000000000000000000000000000000000000000000000000000006000000000000000000000000000000000000000000088923
:3D6DD9000000000000000000000000000000000000000000000000000000000000000000000000000006000000000000000000000000000000000000000000808176
:3D6E160000000000000000000000000000000000000000000000000000000000000000000000000000060000000000000000000000000000000000000000000889A8
:3D6E53000200000000000000000000000000000000000000000000000000000000000000000000000006000000000000000000000000000000000000000000088B67
:3D6E9000020000000000000000000000000000000000000000000000000000000000000000000000000000000000000000000000000000000000000000000090F43F
:3D6ECD00020000000000000000000000000000000000000000000000000000000000000000000000000000000000000000000000000000000000000000000008ED91
:3D6F0A00020000000000000000000000000000000000000000000000000000000000000000000000000000000000000000000000000000000000000000000008ED53
:3D6F4700000000000000000000000000000000000000000000000000000000000000000000000000000000000000000000000000000000000000000000000008EF16
:3D6F8400000000000000000000000000000000000000000000000000000000000000000000000000000000000000000000000000000000000000000000000080E769
:3D6FC100000000000000000000000000000000000000000000000000000000000000000000000000000000000000000000000000000000000000000000000080E72C
:3D6FFE00000000000000000000000000000000000000000000000000000000000000000000000000000000000000000000000000000000000000000000000080E7EF
:3D703B00000000000000000000000000000000000000000000000000000000000000000000000000000000000000000000000000000000000000000000000008EF21
:3D707800020000000000004000000000000000000000000000000000000000000000000000000800000000400000000000000000000000000000000000000088A920
:3D70B500020000000000600000000000000000000000000000000000000000000000000000800100000018000000000000000000000000000000000000000090947F
:3D70F200020000000000000000000000000000000000000000000000000000000000000000000000000000000000000000000000000000000000000000000008ED6A
:3D712F00020000000000400000000000000000000000000000000000000000000000000000000100000010000000000000000000000000000000000000000008AD1B
:3D716C00000000000000800100000000000000000000000000000000000000000000000000000600000060000000000000000000000000000000000000000088F681
:3D71A9001E0000000000800100000000000000000000000000000000000000000000000000000600000060000000000000000000000000000000000000000000E0C4
:3D71E6001E0000000000800100000000000000000000000000000000000000000000000000000600000060000000000000000000000000000000000000000000E087
:3D722300000000000000800100000000000000000000000000000000000000000000000000000600000060000000000000000000000000000000000000000000FE49
:3D726000000110000110000110000110000110000110000110000110000110000000000040000440000440000440000440000440000440000440000440000480E78D
:3D729D00000000000000000000000000000000000000000000000000000000000000000000000000000000000000000000000000000000000000000000000080E74D
:3D72DA00800118800118800118800118800118800118800118800118800118000000000060000660000660000660000660000660000660000660000660000680E719
:3D731700800008800008800008800008800008800008800008800008800008000000000020000220000220000220000220000220000220000220000220000280E7D8
:3D735400000000000000100050000000000000000000000000000000000000000000000000800000002000000400000000000000000000000000000000000000EC0C
:3D739100000000000000000000000000000000000000000000000000000000000000000000000000000000000400000000000000000000000000000000000080A398
:3D73CE00000000000000000000000000000000000000000000000000000000000000000000000000000000000000000000000000000000000000000000000080E71B
:3D740B00000000000000000000000000000000000000000000000000000000000000000000000000000000000000000000000000000000000000000000000080E7DD
:3D744800000000000000100040000000000000000000000000000000000000000000000000800000002000000400000000000000000000000000000000000000FD16
:3D748500000000000000000000000000000000000000000000000000000000000000000000000000000000000000000000000000000000000000000000000080E763
:3D74C200000000000000000000000000000000000000000000000000000000000000000000000000000000000000000000000000000000000000000000000028CD98
:3D74FF00000000000000000000000000000000000000000000000000000000000000000000000000008000000000000000000000000000000000000000000008E7E1
:3D753C00000000008000001000000000000000000000000000000000000000000000000000000000000000000200000000000000000000000000000000000080CC34
:3D757900000000000000000010000000000000000000000000000000000000000000000000000100000000000000000000000000000000000000000000000080E75D
:3D75B600000000000000020000000000000000000000000000000000000000000000000000000000000000400000000000000000000000000000000000000080A531
:3D75F300000000000000000000000000000000000000000000000000000000000000000000000000000000000000000000000000000000000000000000000080E7F4
:3D763000000000000000000000000000000000000000000000000000000000000000000000000000000000000000000000000000000000000000000000000080E7B6
:3D766D00000000000000000000000000000000000000000000000000000000000000000000000000200000000000000000000000000000000000000000000080C779
:3D76AA00000000000000000000000000000000000000000000000000000000000000000000000000000000000000000000000000000000000000000000000080E73C
:3D76E7000000000000000000000000000000000000000000000000000000000000000000000000000000000000000000000000000000000000000000000000F090E6
:3D772400000000000000000000000000000000000000000000000000000000000000000000000000000000000000000000000000000000000000000000000080E7C1
:3D776100000000000000000000000000000000000000000000000000000000000000000000000000000000000000000000000000000000000000000000000080E784
:3D779E00000000000000000000000000000000000000000000000000000000000000000000000000000000000000000000000000000000000000000000000080E747
:3D77DB00000000000000000000000000000000000000000000000000000000000000000000000000000000000000000000000000000000000000000000000080E70A
:3D781800000000000000000000000000000000000000000000000000000000000000000000000000000000000000000000000000000000000000000000000080E7CC
:3D785500000000000000000000000000000000000000000000000000000000000000000000000000000000000000000000000000000000000000000000000080E78F
:3D789200000000000000000000000000000000000000000000000000000000000000000000000000000000000000000000000000000000000000000000000080E752
:3D78CF00000000000000000000000000000000000000000000000000000000000000000000000000000000000000000000000000000000000000000000000080E715
:3D790C00000000000000000000000000000000000000000000000000000000000000000000000000000000000000000000000000000000000000000000000080E7D7
:3D794900000000000000000000000000000000000000000000000000000000000000000000000000000000000000000000000000000000000000000000000080E79A
:3D798600000000000000000000000000000000000000000000000000000000000000000000000000000000000000000000000000000000000000000000000080E75D
:3D79C300000000000000000000000000000000000000000000000000000000000000000000000000000000000000000000000000000000000000000000000080E720
:3D7A00000000000000000000000000000000000000000000000000000000000000000000000000000000000000000000000000000000000000000000000000C0A3E6
:3D7A3D00000000000000000000000000000000000000000000000000000000000000000000000000000000000000000000000000000000000000000000000080E7A5
:3D7A7A00000000000000000000000000000000000000000000000000000000000000000000000000000000000000000000000000000000000000000000000080E768
:3D7AB7000000000000000000000000000000000000000000000000000000000000000000000000000000000000000000000000000000000000000000000000A0C52D
:3D7AF400000000000000000000000000000000000000000000000000000000000000000000000000000000000000000000000000000000000000000000000080E7EE
:3D7B3100000000000000000000000000000000000000000000000000000000000000000000000000000000000000000000000000000000000000000000000090F691
:3D7B6E00000000000000000000000000000000000000000000000000000000000000000000000000000000000000000000000000000000000000000000000080E773
:3D7BAB00000000000000000000000000000000000000000000000000000000000000000000000000000000000000000000000000000000000000000000000080E736
:3D7BE800000000000000000000000000000000000000000000000000000000000000000000000000000000000000000000000000000000000000000000000080E7F9
:3D7C2500000000000000000000000000000000000000000000000000000000000000000000000000000000000000000000000000000000000000000000000080E7BB
:3D7C6200000000000000000000000000000000000000000000000000000000000000000000000000000000000000000000000000000000000000000000000080E77E
:3D7C9F00000000000000000000000000000000000000000000000000000000000000000000000000000000000000000000000000000000000000000000000080E741
:3D7CDC00000000000000000000000000000000000000000000000000000000000000000000000000000000000000000000000000000000000000000000000080E704
:3D7D1900000000000000000000000000000000000000000000000000000000000000000000000000000000000000000000000000000000000000000000000080E7C6
:3D7D5600000000000000000000000000000000000000000000000000000000000000000000000000000000000000000000000000000000000000000000000080E789
:3D7D9300000000000000000000000000000000000000000000000000000000000000000000000000000000000000000000000000000000000000000000000008EFBC
:3D7DD000000000000000000000000000000000000000000000000000000000000000000000000000000000000000000000000000000000000000000000000080E70F
:3D7E0D00000000000000000000000000000000000000000000000000000000000000000000000000000000000000000000000000000000000000000000000080E7D1
:3D7E4A00000000000000000000000000000000000000000000000000000000000000000000000000000000000000000000000000000000000000000000000080E794
:3D7E870000000000000000000000000000000000000000000000000000000000000000000000000000000000000000000000000000000000000000000000006889CD
:3D7EC400000000000000000000000000000000000000000000000000000000000000000000000000000000000000000000000000000000000000000000000080E71A
:3D7F01000000000000000000000000000100400000000000000000000000000000000000000000000000000000000000080000000000020000000000000000008A6E
:3D7F3E00000000000000000000000000000000000000000000000000000000000000000000000000000000000000000000000000000000000000000000000080E79F
:3D7F7B00000000000000000000000000000000000000000000000000000000000000000000000000000000000000000000000000000000000000000000000080E762
:3D7FB800000000000000000000000000000000000000000000000000000000000000000000000000000000000000000000000000000000000000000000000080E725
:3D7FF5000000000000000000000000000300500000000000000000000000000000000000000000000000000000000000080000000000030000000000000000008968
:3D803200000110000110000110000110000110000110000110000110000110000000000040000440000440000440000440000440000440000440000440000480E7AD
:3D806F00000000000000000000000000000000000000000000000000000000000000000000000000000000000000000000000000000000000000000000000080E76D
:3D80AC00800118800118800118800118800118800118800118800118800118000000000060000660000660000660000660000660000660000660000660000608EFA9
:3D80E900820008800008800008800008800008800008800008800008800008000000000020000220000220000220000220000220000220000220000220000208ED69
:3D812600020000000000000000000000000000000000000000000000000000000000000000000000000000000000000000000000000000000000000000000090F496
:3D816300020000000000000000000000000000000000000000000000000000000000000000000000000000000000000000000000000000000000000000000008EDE8
:3D81A000020000000000000000000000000000000000000000000000000000000000000000000000000000000000000000000000000000000000000000000008EDAB
:3D81DD00000000000000000000000000000000000000000000000000000000000000000000000000000000000000000000000000000000000000000000000008EF6E
:3D821A00000000000000000000000000000000000000000000000000000000000000000000000000000000000000000000000000000000000000000000000080E7C0
:3D825700000000000000000000000000000000000000000000000000000000000000000000000000000000000000000000000000000000000000000000000080E783
:3D829400000000000000000000000000000000000000000000000000000000000000000000000000000000000000000000000000000000000000000000000080E746
:3D82D100000000000000000000000000000000000000000000000000000000000000000000000000000000000000000000000000000000000000000000000008EF79
:3D830E00020000000000000000000000000000000000000000000000000000000000000000000000000000000000000000000000000000000000000000000008ED3B
:3D834B00020000000000000000000000000000000000000000000000000000000000000000000000000000000000000000000098400000000000000000000090ADDE
:3D838800020000000000000000000000000000000000000000000000000000000000000000000000000000000000000000000000000000000000000000000008EDC1
:3D83C500020000000000000000000000000000000000000000000000000000000000000000000000000000000000000000000010000000000000000000000008FC65
:3D840200000000000000000000000000000000000000000000000000000000000000000000000000000000000000000000000060000000000000000000000008894C
:3D843F00000000000000000000000000000000000000000000000000000000000000000000000000000000000000000000000060000000000000000000000080819F
:3D847C0000000000000000000000000000000000000000000000000000000000000000000000000000000000000000000000006000000000000000000000000889D2
:3D84B9000200000000000000000000000000000000000000000000000000000000000000000000000000000000000000000000600000000000000000000000088B91
:3D84F600020000000000000000008000000000000000000000000000000000000000000000000000000000000000000000000000000000000000000000000090FC3B
:3D8533000200000000000000006000000000000000000000000000000000000000000000000000000000000000000000000000000000000000000000000000088D14
:3D857000020000000000000000000000000000000000000000000000000000000000000000000000000000000000000000000000000000000000000000000008EDD7
:3D85AD00000000000000000000400000000000000000000000000000000000000000000000000000000000000000000000000000000000000000000000000008AF9A
:3D85EA00000000000000000000800100000000000000000000000000000000000000000000000000000000000000000000000000000000000000000000000000FED5
:3D862700000000000000000000800100000000000000000000000000000000000000000000000000000000000000000000000000000000000000000000000000FE97
:3D866400000000000000000000800100000000000000000000000000000000000000000000000000000000000000000000000000000000000000000000000000FE5A
:3D86A100000000000000000000800100000000000000000000000000000000000000000000000000000000000000000000000000000000000000000000000088F69D
:3D86DE00020000000000000000000000001000000000000000000000000000000000000000000000000000000000000080000000000000000000000000000088EC59
:3D871B00020000000000000000000000600200000000000000000000000000000000000000000000000000000000000018000000000000000000000000000010AFE6
:3D875800020000000000000000000000000000000000000000000000000000000000000000000000000000000000000000000000000000000000000000000008EDED
:3D879500020000000000000000000000400000000000000000000000000000000000000000000000000000000000000010000000000000000000000000000008BC91
:3D87D2000000000000000000000000008001000000000000000000000000000000000000000000000000000000000000600000000000000000000000000000889071
:3D880F0000000000000000000000000080010000000000000000000000000000000000000000000000000000000000006000000000000000000000000000000098B3
:3D884C0000000000000000000000000080010000000000000000000000000000000000000000000000000000000000006000000000000000000000000000008890F6
:3D88890002000000000000000000000080010000000000000000000000000000000000000000000000000000000000006000000000000000000000000000008892B5
:3D88C600020000000000000000000000000000000000000000000000000000000000000000000000000000000000000800000000000000000000000000000010F467
:3D890300020000000000000000000000000000000000000000000000000000000000000000000000000000000000800900000000000000000000000000000008F4B0
:3D894000020000000000000000000000000000000000000000000000000000000000000000000000000000000000000000000000000000000000000000000008ED03
:3D897D00000000000000000000000000000000000000000000000000000000000000000000000000000000000000000100000000000000000000000000000008FEB6
:3D89BA000000000000000000000000000000000000000000000000000000000000000000000000000000000000000006000000000000000000000000000000808179
:3D89F700000000000000000000000000000000000000000000000000000000000000000000000000000000000000000600000000000000000000000000000080813C
:3D8A340000000000000000000000000000000000000000000000000000000000000000000000000000000000000000060000000000000000000000000000008081FE
:3D8A71000000000000000000000000000000000000000000000000000000000000000000000000000000000000000006000000000000000000000000000000088931
:3D8AAE00020000000000000000000000000000000000000000000000000000000000000000000000000000000000000000000000000000000000000000000008ED94
:3D8AEB000200000000000000000000000000060800000000000000000000000000000000000000000000000000000000000000000000000000000000000000909C12
:3D8B2800020000000000000000000000000000000000000000000000000000000000000000000000000000000000000000000000000000000000000000000008ED19
:3D8B6500020000000000000000000000000004000000000000000000000000000000000000000000000000000000000000000000000000000000000000000008AD18
:3D8BA200000000000000000000000000000018000000000000000000000000000000000000000000000000000000000000000000000000000000000000000088F600
:3D8BDF00000000000000000000000000000018000000000000000000000000000000000000000000000000000000000000000000000000000000000000000000FE43
:3D8C1C00000000000000000000000000000018000000000000000000000000000000000000000000000000000000000000000000000000000000000000000000FE05
:3D8C5900020000000000000000000000000018000000000000000000000000000000000000000000000000000000000000000000000000000000000000000088F448
:3D8C9600020000000000000000000000000000000000000000000000000000000000000000000000000000000000000000000000000000000000000000000008EDAA
:3D8CD300020000000000000000000000000000000000000000000000000000000000000000000000000000000000000000000000000000000000000000000008ED6D
:3D8D1000020000000000000000000000000000000000000000000000000000000000000000000000000000000000000000000000000000000000000000000008ED2F
:3D8D4D00000000000000000000000000000000000000000000000000000000000000000000000000000000000000000000000000000000000000000000000080E782
:3D8D8A00000000000000000000000000000000000000000000000000000000000000000000000000000000000000000000000000000000000000000000000080E745
:3D8DC700000000000000000000000000000000000000000000000000000000000000000000000000000000000000000000000000000000000000000000000080E708
:3D8E0400000000000000000000000000000000000000000000000000000000000000000000000000000000000000000000000000000000000000000000000080E7CA
:3D8E4100000000000000000000000000000000000000000000000000000000000000000000000000000000000000000000000000000000000000000000000080E78D
:3D8E7E00020000000000000000000000000000000001000000000000000000000000000000000000000000000000400000000000000000000000000000000008BDAF
:3D8EBB00020000000000000000000006010000600000000000000000000000000000000000000000000000000098000000800902000000000000000000000008CC1A
:3D8EF800020000000000000000000000000000000000000000000000000000000000000000000000000000000000000000000000000000000000000000000008ED46
:3D8F3500020000000000000000000004000000400000000000000000000000000000000000000000000000000010000000000100000000000000000000000008EDB3
:3D8F7200000000000000000000000018000000800100000000000000000000000000000000000000000000000060000000000600000000000000000000000080E75C
:3D8FAF001E0000000000000000000018000000800100000000000000000000000000000000000000000000000060000000000600000000000000000000000080F9EF
:3D8FEC001E0000000000000000000018000000800100000000000000000000000000000000000000000000000060000000000600000000000000000000000018E033
:3D902900000000000000000000000018000000800100000000000000000000000000000000000000000000000060000000000600000000000000000000000080E7A4
:3D906600000110000110000110000110000110000110000110000110000110000000000040000440000440000440000440000440000440000440000440000480E769
:3D90A300000000000000000000000000000000000000000000000000000000000000000000000000000000000000000000000000000000000000000000000080E729
:3D90E000800118800118800118800118800118800118800118800118800118000000000060000660000660000660000660000660000660000660000660000680E7F5
:3D911D00800008800008800008800008800008800008800008800008800008000000000020000220000220000220000220000220000220000220000220000280E7B4
:3D915A00000000000000000000000000000000010000000000000000000000000000000000000000000000000000000002000000000000000000000000000080C68F
:3D919700000000000000000000000000000000000000000000000000000000000000000000000000000000000000000000000000000000000000000000000080E734
:3D91D400000000000000000000000000000000000000000000000000000000000000000000000000000000000000000000000000000000000000000000000080E7F7
:3D921100000000000000000000000000000000800000000000000000000000000000000000000000000000000020000000000200000000000000000000000000EF8F
:3D924E00000000000000000000000008000000010000000000000000000000000000000000000000000000000000000002000000000000000000000000000000CE0A
:3D928B00000000000000000000000000000000000000000000000000000000000000000000000000000000000000000000000000000000000000000000000080E73F
:3D92C8000000000000000000000000000000000000000000000000000000000000000000000000000000000000000000000000000000000000000000000000C0A306
:3D930500000000000000000000000000000000020000000000000000000000000000000000000000000000000000000000000000000000000000000000000080E5C4
:3D934200000000000000000000000000800000000000000000000000000000000000000000000000000000000000200000000000000000000000000000000000CF7F
:3D937F00000000000000000000000010000000000000000000000000000000000000000000000000000000000000000010000001000000000000000000000080F719
:3D93BC000000000000000000000020000000000000010000000000000000000000000000000000000000000000000001000000000000000000000000000000C0A0F2
:3D93F900000000000000000000000000000000000000000000000000000000000000000000000000000000000000000000000000000000000000000000000080E7D0
:3D943600000000000000000000000000000000000000000000000000000000000000000000000000000000000000000000000000000000000000000000000080E792
:3D947300000000000000000000000000000000000000000000000000000000000000000000000000000000000000000000000000200000000000000000000080C755
:3D94B000000000000000000000000000000000000000000000000000000000000000000000000000000000000000000000000000000000000000000000000080E718
:3D94ED00000000000000000000000000000000000000000000000000000000000000000000000000000000000000000000000000000000000000000000000080E7DB
:3D952A000000000000000000000000000000000000000000000000000000000000000000000000000000000000000000000000000000000000000000000000A0C59F
:3D956700000000000000000000000000000000000000000000000000000000000000000000000000000000000000000000000000000000000000000000000080E760
:3D95A400000000000000000000000000000000000000000000000000000000000000000000000000000000000000000000000000000000000000000000000080E723
:3D95E100000000000000000000000000000000000000000000000000000000000000000000000000000000000000000000000000000000000000000000000080E7E6
:3D961E00000000000000000000000000000000000000000000000000000000000000000000000000000000000000000000000000000000000000000000000080E7A8
:3D965B00000000000000000000000000000000000000000000000000000000000000000000000000000000000000000000000000000000000000000000000080E76B
:3D969800000000000000000000000000000000000000000000000000000000000000000000000000000000000000000000000000000000000000000000000080E72E
:3D96D500000000000000000000000000000000000000000000000000000000000000000000000000000000000000000000000000000000000000000000000080E7F1
:3D971200000000000000000000000000000000000000000000000000000000000000000000000000000000000000000000000000000000000000000000000080E7B3
:3D974F00000000000000000000000000000000000000000000000000000000000000000000000000000000000000000000000000000000000000000000000080E776
:3D978C00000000000000000000000000000000000000000000000000000000000000000000000000000000000000000000000000000000000000000000000080E739
:3D97C900000000000000000000000000000000000000000000000000000000000000000000000000000000000000000000000000000000000000000000000080E7FC
:3D980600000000000000000000000000000000000000000000000000000000000000000000000000000000000000000000000000000000000000000000000080E7BE
:3D984300000000000000000000000000000000000000000000000000000000000000000000000000000000000000000000000000000000000000000000000080E781
:3D988000000000000000000000000000000000000000000000000000000000000000000000000000000000000000000000000000000000000000000000000080E744
:3D98BD00000000000000000000000000000000000000000000000000000000000000000000000000000000000000000000000000000000000000000000000080E707
:3D98FA00000000000000000000000000000000000000000000000000000000000000000000000000000000000000000000000000000000000000000000000090F6AB
:3D9937000000000000000000000000000000000000000000000000000000000000000000000000000000000000000000000000000000000000000000000000E08192
:3D997400000000000000000000000000000000000000000000000000000000000000000000000000000000000000000000000000000000000000000000000080E74F
:3D99B100000000000000000000000000000000000000000000000000000000000000000000000000000000000000000000000000000000000000000000000080E712
:3D99EE00000000000000000000000000000000000000000000000000000000000000000000000000000000000000000000000000000000000000000000000080E7D5
:3D9A2B00000000000000000000000000000000000000000000000000000000000000000000000000000000000000000000000000000000000000000000000080E797
:3D9A6800000000000000000000000000000000000000000000000000000000000000000000000000000000000000000000000000000000000000000000000080E75A
:3D9AA500000000000000000000000000000000000000000000000000000000000000000000000000000000000000000000000000000000000000000000000008EF8D
:3D9AE200000000000000000000000000000000000000000000000000000000000000000000000000000000000000000000000000000000000000000000000080E7E0
:3D9B1F00000000000000000000000000000000000000000000000000000000000000000000000000000000000000000000000000000000000000000000000080E7A2
:3D9B5C00000000000000000000000000000000000000000000000000000000000000000000000000000000000000000000000000000000000000000000000080E765
:3D9B9900000000000000000000000000000000000000000000000000000000000000000000000000000000000000000000000000000000000000000000000080E728
:3D9BD600000000000000000000000000000000000000000000000000000000000000000000000000000000000000000000000000000000000000004000000080E3AF
:3D9C1300000000000000000000000000000000000000000000000000000000000000000000000000000000000000000000000000000000000000000000000080E7AD
:3D9C5000000000000000000000000000000000000000000000000000000000000000000000000000000000000000000000000000000000000000000000000080E770
:3D9C8D000000000000000000000000000000000000000000000000000000000000000000000000000000000000000000000000000000000020000000000000A0C713
:3D9CCA00000000000000000000000000000000000000000000000000000000000000000000000000000000000000000000000000000000000000000000000080E7F6
:3D9D0700000000000000000000000000000000000000000000500000000000000000000000000000000000000000000000000000000000002800000000000000B5F2
:3D9D4400000000000000000000000000000000000000000000000000000000000000000000000000000000000000000000000000000000000000000000000080E77B
:3D9D8100000000000000000000000000000000000000000000000000000000000000000000000000000000000000000000000000000000000000000000000080E73E
:3D9DBE00100000000000000000000000000000000000000000000000000000000000000000000000000000000000000000000000000000000000000000000080F7E1
:3D9DFB0000000000000000000000000000000000000000000054000000000000000000000000000000000000000000000000000000000000A800000000000000B976
:3D9E3800000110000110000110000110000110000110000110000110000110000000000040000440000440000440000440000440000440000440000440000480E789
:3D9E7500000000000000000000000000000000000000000000000000000000000000000000000000000000000000000000000000000000000000000000000080E749
:3D9EB200800118800118800118800118800118800118800118800118800118000000000060000660000660000660000660000660000660000660000660000608EF85
:3D9EEF00820008800008800008800008800008800008800008800008800008000000000020000220000220000220000220000220000220000220000220000208ED45
:3D9F2C00020000000000000000000000000000000000000000000000000000000000000000000000000000000000000000000000000000000000000000000090F472
:3D9F6900020000000000000000000000000000000000000000000000000000000000000000000000000000000000000000000000000000000000000000000008EDC4
:3D9FA600020000000000000000000000000000000000000000000000000000000000000000000000000000000000000000000000000000000000000000000008ED87
:3D9FE300000000000000000000000000000000000000000000000000000000000000000000000000000000000000000000000000000000000000000000000008EF4A
:3DA02000000000000000000000000000000000000000000000000000000000000000000000000000000000000000000000000000000000000000000000000080E79C
:3DA05D00000000000000000000000000000000000000000000000000000000000000000000000000000000000000000000000000000000000000000000000080E75F
:3DA09A00000000000000000000000000000000000000000000000000000000000000000000000000000000000000000000000000000000000000000000000080E722
:3DA0D700000000000000000000000000000000000000000000000000000000000000000000000000000000000000000000000000000000000000000000000008EF55
:3DA11400020000000000000000000000000000000000000001000000000000000000000000000000000000000000000000000000000000000000000000000008FD06
:3DA15100020000000000000000000000000000000000600000000000000000000000000000000000000000000000000000000000000000000000000000000090944B
:3DA18E00020000000000000000000000000000000000000000000000000000000000000000000000000000000000000000000000000000000000000000000008ED9D
:3DA1CB00020000000000000000000000000000000000400000000000000000000000000000000000000000000000000000000000000000000000000000000008AD60
:3DA20800000000000000000000000000000000000000800100000000000000000000000000000000000000000000000000000000000000000000000000000088F61A
:3DA24500000000000000000000000000000000000000800100000000000000000000000000000000000000000000000000000000000000000000000000000000FE5D
:3DA28200000000000000000000000000000000000000800100000000000000000000000000000000000000000000000000000000000000000000000000000088F6A0
:3DA2BF00020000000000000000000000000000000000800100000000000000000000000000000000000000000000000000000000000000000000000000000088F463
:3DA2FC00020000000000000000000000000000000000000000000000000000000000000000000000000000000000000000000000000000200000000000000090D49F
:3DA33900020000000000000000000000000000000000000000000000000000000000000000000000000000000000000000000000000018800901000000000088FDBE
:3DA37600020000000000000000000000000000000000000000000000000000000000000000000000000000000000000000000000000000000000000000000008EDB3
:3DA3B300000000000000000000000000000000000000000000000000000000000000000000000000000000000000000000000000000010000100000000000008EF65
:3DA3F000000000000000000000000000000000000000000000000000000000000000000000000000000000000000000000000000000060000600000000000080E763
:3DA42D00000000000000000000000000000000000000000000000000000000000000000000000000000000000000000000000000000060000600000000000080E725
:3DA46A00000000000000000000000000000000000000000000000000000000000000000000000000000000000000000000000000000060000600000000000080E7E8
:3DA4A700000000000000000000000000000000000000000000000000000000000000000000000000000000000000000000000000000060000600000000000008EF1B
:3DA4E400020000000000000000000000000000000000000000001000000000000000000000000000000000000000000000000000000000000000000000000008EC35
:3DA52100020000000000000000000000000000000000000000600200000000000000000000000000000000000000000000000000000000000000000000000090B653
:3DA55E00020000000000000000000000000000000000000000000000000000000000000000000000000000000000000000000000000000000000000000000008EDC9
:3DA59B00020000000000000000000000000000000000000000400000000000000000000000000000000000000000000000000000000000000000000000000008AD8C
:3DA5D800000000000000000000000000000000000000000000800100000000000000000000000000000000000000000000000000000000000000000000000088F647
:3DA61500000000000000000000000000000000000000000000800100000000000000000000000000000000000000000000000000000000000000000000000000FE89
:3DA65200000000000000000000000000000000000000000000800100000000000000000000000000000000000000000000000000000000000000000000000088F6CC
:3DA68F00020000000000000000000000000000000000000000800100000000000000000000000000000000000000000000000000000000000000000000000088F48F
:3DA6CC00020000000000000000000000000000000000000000000000000000000000000000000000000000000000000000000000000000000000000000000090F4CB
:3DA70900020000000000000000000000000000000000000000000000000000000000000000000000000000000000000000000000800902000000000000000008D4AA
:3DA74600020000000000000000000000000000000000000000000000000000000000000000000000000000000000000000000000000000000000000000000008EDDF
:3DA78300000000000000000000000000000000000000000000000000000000000000000000000000000000000000000000000000000100000000000000000008FE92
:3DA7C0000000000000000000000000000000000000000000000000000000000000000000000000000000000000000000000000000006000000000000000000808155
:3DA7FD000000000000000000000000000000000000000000000000000000000000000000000000000000000000000000000000000006000000000000000000808118
:3DA83A0000000000000000000000000000000000000000000000000000000000000000000000000000000000000000000000000000060000000000000000008081DA
:3DA87700000000000000000000000000000000000000000000000000000000000000000000000000000000000000000000000000000600000000000000000008890D
:3DA8B400020000000000000000000000000000000000000000000000000000000000000000000000000000000000000000000000000000000000000000000008ED70
:3DA8F100020000000000000000000000000000000000000000000000000000000000000000000000000000000000000000000000000000000000000000000090F4A4
:3DA92E00020000000000000000000000000000000000000000000000000000000000000000000000000000000000000000000000000000000000000000000008EDF5
:3DA96B00020000000000000000000000000000000000000000000000000000000000000000000000000000000000000000000000000000000000000000000008EDB8
:3DA9A800000000000000000000000000000000000000000000000000000000000000000000000000000000000000000000000000000000000000000000000008EF7B
:3DA9E500000000000000000000000000000000000000000000000000000000000000000000000000000000000000000000000000000000000000000000000080E7CE
:3DAA2200000000000000000000000000000000000000000000000000000000000000000000000000000000000000000000000000000000000000000000000008EF00
:3DAA5F00020000000000000000000000000000000000000000000000000000000000000000000000000000000000000000000000000000000000000000000008EDC3
:3DAA9C00020000000000000000000000000000000000000020000000000000000000000000000000000000000000000000000000000000000000000000000090D6F5
:3DAAD900020000000000000000000000000000000000000006000000000000000000000000000000000000000000000000000000000000000098400000000008D484
:3DAB1600020000000000000000000000000000000000000000000000000000000000000000000000000000000000000000000000000000000000000000000008ED0B
:3DAB5300000000000000000000000000000000000000000004000000000000000000000000000000000000000000000000000000000000000010000000000008BEEB
:3DAB90000000000000000000000000000000000000000000180000000000000000000000000000000000000000000000000000000000000000600000000000009878
:3DABCD00000000000000000000000000000000000000000018000000000000000000000000000000000000000000000000000000000000000060000000000000983B
:3DAC0A0000000000000000000000000000000000000000001800000000000000000000000000000000000000000000000000000000000000006000000000000098FD
:3DAC470000000000000000000000000000000000000000001800000000000000000000000000000000000000000000000000000000000000006000000000000098C0
:3DAC8400020000000000000000000000000000000000000000000000000000000000000000000000000000000000000000000000000000000000000001000008FD8B
:3DACC100020000000000000000000000000000000006010000000006080000000000000000000000000000000000000000000000000000000000800100000088FD39
:3DACFE00020000000000000000000000000000000000000000000000000000000000000000000000000000000000000000000000000000000000000000000008ED22
:3DAD3B00020000000000000000000000000000000004000000000004000000000000000000000000000000000000000000000000000000000000000100000008FCCC
:3DAD78000000000000000000000000000000000000180000000000180000000000000000000000000000000000000000000000000000000000000006000000808167
:3DADB5001E00000000000000000000000000000000180000000000180000000000000000000000000000000000000000000000000000000000000006000000809FEE
:3DADF2000E00000000000000000000000000000000180000000000180000000000000000000000000000000000000000000000000000000000000006000000088751
:3DAE2F0000000000000000000000000000000000001800000000001800000000000000000000000000000000000000000000000000000000000000060000008081AF
:3DAE6C00000110000110000110000110000110000110000110000110000110000000000040000440000440000440000440000440000440000440000440000480E745
:3DAEA900000000000000000000000000000000000000000000000000000000000000000000000000000000000000000000000000000000000000000000000080E705
:3DAEE600800118800118800118800118800118800118800118800118800118000000000060000660000660000660000660000660000660000660000660000680E7D1
:3DAF2300800008800008800008800008800008800008800008800008800008000000000020000220000220000220000220000220000220000220000220000280E790
:3DAF600000000000000000000000000000000000000000004000000000000000000000000000000000000000000000000000000000000200000000A00000008089C9
:3DAF9D00000000000000000000000000000000000000000000000000000000000000000000000000000000000000000000000000000000000000000000000080E710
:3DAFDA00000000000000000000000000000000000000000000000000000000000000000000000000000000000000000000000000000000000000000000000080E7D3
:3DB01700000000000000000000000000000000000008000000000008000000000000000000000000000000000000000000000000000000000000000200000080C5A5
:3DB05400000000000000000000000000000000000000000040000000000000000000000000000000000000000000000000000000000002000000002000000080815C
:3DB09100000000000000000000000000000000000000000000000000000000000000000000000000000000000000000000000000000000000000000000000080E71B
:3DB0CE000000000000000000000000000000000000000000000000000000000000000000000000000000000000000000000000000000000000000000000000B0D4C1
:3DB10B00000000000000000000000000000000000000000000000000020000000000000000000000000000000000000000000000000000000000000000000080E5A0
:3DB14800000000000000000000000000000000000000000000800000000000000000000000000000000000000000000000000000000000000000000000000000EF5B
:3DB18500000000000000000000000000000000000010000004000000000000000000000000000000000000000000000000000000000001000000000000000080A652
:3DB1C2000000000000000000000000000000000000000000010000000000000000000000000000000000000000000000000000000000000800000000000000A0DDCA
:3DB1FF00000000000000000000000000000000000000000000000000000000000000000000000000000000000000000000000000000000000000000000000080E7AC
:3DB23C00000000000000000000000000000000000000000000000000000000000000000000000000000000000000000000000000000000000000000000000080E76E
:3DB27900000000000000000000000000000000000000000000000000000000000000000000000000000000000000000000000000000000000000200000000080C731
:3DB2B6000000000000000000000000000000000000000000000000000000000000000000000000000000000000000000000000000000000000000000000000C0A3F8
:3DB2F300000000000000000000000000000000000000000000000000000000000000000000000000000000000000000000000000000000000000000000000080E7B7
:3DB33000000000000000000000000000000000000000000000000000000000000000000000000000000000000000000000000000000000000000000000000090F65A
:3DB36D00000000000000000000000000000000000000000000000000000000000000000000000000000000000000000000000000000000000000000000000080E73C
:3DB3AA00000000000000000000000000000000000000000000000000000000000000000000000000000000000000000000000000000000000000000000000080E7FF
:3DB3E700000000000000000000000000000000000000000000000000000000000000000000000000000000000000000000000000000000000000000000000080E7C2
:3DB42400000000000000000000000000000000000000000000000000000000000000000000000000000000000000000000000000000000000000000000000080E784
:3DB46100000000000000000000000000000000000000000000000000000000000000000000000000000000000000000000000000000000000000000000000080E747
:3DB49E00000000000000000000000000000000000000000000000000000000000000000000000000000000000000000000000000000000000000000000000080E70A
:3DB4DB00000000000000000000000000000000000000000000000000000000000000000000000000000000000000000000000000000000000000000000000080E7CD
:3DB51800000000000000000000000000000000000000000000000000000000000000000000000000000000000000000000000000000000000000000000000080E78F
:3DB55500000000000000000000000000000000000000000000000000000000000000000000000000000000000000000000000000000000000000000000000080E752
:3DB59200000000000000000000000000000000000000000000000000000000000000000000000000000000000000000000000000000000000000000000000080E715
:3DB5CF00000000000000000000000000000000000000000000000000000000000000000000000000000000000000000000000000000000000000000000000018FE29
:3DB60C000000000000000000000000000000000000000000000000000000000000000000000000000000000000000000000000000000000000000000000000C0A39E
:3DB64900000000000000000000000000000000000000000000000000000000000000000000000000000000000000000000000000000000000000000000000080E75D
:3DB68600000000000000000000000000000000000000000000000000000000000000000000000000000000000000000000000000000000000000000000000080E720
:3DB6C300000000000000000000000000000000000000000000000000000000000000000000000000000000000000000000000000000000000000000000000080E7E3
:3DB70000000000000000000000000000000000000000000000000000000000000000000000000000000000000000000000000000000000000000000000000080E7A5
:3DB73D00000000000000000000000000000000000000000000000000000000000000000000000000000000000000000000000000000000000000000000000080E768
:3DB77A00000000000000000000000000000000000000000000000000000000000000000000000000000000000000000000000000000000000000000000000080E72B
:3DB7B700000000000000000000000000000000000000000000000000000000000000000000000000000000000000000000000000000000000000000000000080E7EE
:3DB7F400000000000000000000000000000000000000000000000000000000000000000000000000000000000000000000000000000000000000000000000080E7B1
:3DB831000000000000000000000000000000000000000000000000000000000000000000000000000000000000000000000000000000000000000000000000A0C575
:3DB86E00000000000000000000000000000000000000000000000000000000000000000000000000000000000000000000000000000000000000000000000080E736
:3DB8AB00000000000000000000000000000000000000000000000000000000000000000000000000000000000000000000000000000000000000000000000080E7F9
:3DB8E800000000000000000000000000000000000000000000000000000000000000000000000000000000000000000000000000000000000000000000000080E7BC
:3DB92500000000000000000000000000000000000000000000000000000000000000000000000000000000000000000000000000000000000000000000000080E77E
:3DB96200000000000000000000000000000000000000000000000000000000000000000000000000000000000000000000000000000000000000000000000080E741
:3DB99F00000000000000000000000000000000000000000000000000000000000000000000000000000000000000000000000000000000000000000000000080E704
:3DB9DC00000000000000000000000000000000000000000000000000000000000000000000000000000000000000000000000000000000000000000000000080E7C7
:3DBA1900000000000000000000000000000000000000000000000000000000000000000000000000000000000000000000000000000000000000000000000080E789
:3DBA5600000000000000000000000000000000000000000000000000000000000000000000000000000000000000000000000000000000000000000000000080E74C
:3DBA93000000000000000000000000000000000000000000000000000000000000000000000000000000000000000000000000000000000000000000000000688985
:3DBAD000000000000000000000000000000000000000000000000000000000000000000000000000000000000000000000000000000000000000000000000080E7D2
:3DBB0D000000040000000000000000000000000000000000000000000000000100000000000000020000000000000000000000000000000000000000000008008666
:3DBB4A00000000000000000000000000000000000000000000000000000000000000000000000000000000000000000000000000000000000000000000000080E757
:3DBB8700000000000000000000000000000000000000000000000000000000000000000000000000000000000000000000000000000000000000000000000080E71A
:3DBBC400000000000000000000000000000000000000000000000000000000000000000000000000000000000000000000000000000000000000000000000080E7DD
:3DBC01000000040000000000000000000000000000000000000000000000000100000000000000030000000000000000000000000000000000000000000008009660
:3DBC3E00000110000110000110000110000110000110000110000110000110000000000040000440000440000440000440000440000440000440000440000480E765
:3DBC7B00000000000000000000000000000000000000000000000000000000000000000000000000000000000000000000000000000000000000000000000080E725
:3DBCB800800118800118800118800118800118800118800118800118800118000000000060000660000660000660000660000660000660000660000660000608EF61
:3DBCF500820008800008800008800008800008800008800008800008800008000000000020000220000220000220000220000220000220000220000220000208ED21
:3DBD3200020000000000000000000000000000000000000000000000000000000000000000000000000000000000000000000000000000000000000000000090F44E
:3DBD6F00020000000000000000000000000000000000000000000000000000000000000000000000000000000000000000000000000000000000000000000008EDA0
:3DBDAC00020000000000000000000000000000000000000000000000000000000000000000000000000000000000000000000000000000000000000000000008ED63
:3DBDE900000000000000000000000000000000000000000000000000000000000000000000000000000000000000000000000000000000000000000000000008EF26
:3DBE2600000000000000000000000000000000000000000000000000000000000000000000000000000000000000000000000000000000000000000000000080E778
:3DBE6300000000000000000000000000000000000000000000000000000000000000000000000000000000000000000000000000000000000000000000000080E73B
:3DBEA000000000000000000000000000000000000000000000000000000000000000000000000000000000000000000000000000000000000000000000000080E7FE
:3DBEDD00000000000000000000000000000000000000000000000000000000000000000000000000000000000000000000000000000000000000000000000008EF31
:3DBF1A00020000000000000000000000000000000000000000000000000000010000000000000000000000000000000000000000000000000000000000000008ECF3
:3DBF5700020000000000000000000000000000000000000000000000000026000000000018100000000000000000000000000000000000000000000000000010BF8E
:3DBF9400020000000000000000000000000000000000000000000000000000000000000000000000000000000000000000000000000000000000000000000008ED79
:3DBFD100020000000000000000000000000000000000000000000000000004000000000010000000000000000000000000000000000000000000000000000008BC59
:3DC00E000000000000000000000000000000000000000000000000000000180000000000600000000000000000000000000000000000000000000000000000889065
:3DC04B0000000000000000000000000000000000000000000000000000001800000000006000000000000000000000000000000000000000000000000000000098A8
:3DC0880000000000000000000000000000000000000000000000000000001800000000006000000000000000000000000000000000000000000000000000008890EB
:3DC0C50002000000000000000000000000000000000000000000000000001800000000006000000000000000000000000000000000000000000000000000008892AA
:3DC10200020000000000000000000000000000000000000000000000000000000000000000000000000000000000000000000000000000000000000000000094B4B6
:3DC13F00020000000000000000000000000000000000000000000000000000000000000000000000000000000000000000000000000000000000000000800908F43C
:3DC17C00020000000000000000000000000000000000000000000000000000000000000000000000000000000000000000000000000000000000000000000008ED8F
:3DC1B900000000000000000000000000000000000000000000000000000000000000000000000000000000000000000000000000000000000000000000000108FE42
:3DC1F6000000000000000000000000000000000000000000000000000000000000000000000000000000000000000000000000000000000000000000000006808105
:3DC2330000000000000000000000000000000000000000000000000000000000000000000000000000000000000000000000000000000000000000000000068081C7
:3DC27000000000000000000000000000000000000000000000000000000000000000000000000000000000000000000000000000000000000000000000000680818A
:3DC2AD0000000000000000000000000000000000000000000000000000000000000000000000000000000000000000000000000000000000000000000000060889BD
:3DC2EA00020000000000000000000000000000000000000000000000000000000000000000000000000000000000000000000000000000000000000000000008ED20
:3DC32700020026100000000000000000000000000000000000000000000000000000000000000000000000000000000000000000000000000000000000000090A66B
:3DC36400020000000000000000000000000000000000000000000000000000000000000000000000000000000000000000000000000000000000000000000008EDA5
:3DC3A100020004000000000000000000000000000000000000000000000000000000000000000000000000000000000000000000000000000000000000000008ADA4
:3DC3DE00000018000000000000000000000000000000000000000000000000000000000000000000000000000000000000000000000000000000000000000088F68C
:3DC41B00000018000000000000000000000000000000000000000000000000000000000000000000000000000000000000000000000000000000000000000000FECE
:3DC45800000018000000000000000000000000000000000000000000000000000000000000000000000000000000000000000000000000000000000000000088F611
:3DC49500020018000000000000000000000000000000000000000000000000000000000000000000000000000000000000000000000000000000000000000088F4D4
:3DC4D200020000000000000000000000000000000000000000000000000000000000000000000000000000000000000000000000000000000000000000000090F4A7
:3DC50F00020000000000000000000000000000000000000000000000000000000000000000000000000000000000000000000000000000000000000000000008EDF8
:3DC54C00020000000000000000000000000000000000000000000000000000000000000000000000000000000000000000000000000000000000000000000008EDBB
:3DC58900000000000000000000000000000000000000000000000000000000000000000000000000000000000000000000000000000000000000000000000008EF7E
:3DC5C600000000000000000000000000000000000000000000000000000000000000000000000000000000000000000000000000000000000000000000000080E7D1
:3DC60300000000000000000000000000000000000000000000000000000000000000000000000000000000000000000000000000000000000000000000000080E793
:3DC64000000000000000000000000000000000000000000000000000000000000000000000000000000000000000000000000000000000000000000000000080E756
:3DC67D00000000000000000000000000000000000000000000000000000000000000000000000000000000000000000000000000000000000000000000000008EF89
:3DC6BA00020000000000000000000000000000000000000000000000000000000000000000000002000000000000000000000000000000000000000000000008CD6A
:3DC6F700020000000000000000000000000000000000000000000000000000000000000000800100000000000000000000000000000000000000000098200010D4E7
:3DC73400020000000000000000000000000000000000000000000000000000000000000000000000000000000000000000000000000000000000000000000008EDD1
:3DC77100020000000000000000000000000000000000000000000000000000000000000000000100000000000000000000000000000000000000000010000008ED83
:3DC7AE00000000000000000000000000000000000000000000000000000000000000000000000600000000000000000000000000000000000000000060000008EFF1
:3DC7EB00000000000000000000000000000000000000000000000000000000000000000000000600000000000000000000000000000000000000000060000080E744
:3DC82800000000000000000000000000000000000000000000000000000000000000000000000600000000000000000000000000000000000000000060000008EF76
:3DC86500020000000000000000000000000000000000000000000000000000000000000000000600000000000000000000000000000000000000000060000008ED39
:3DC8A200020000000000000000000000000000000000000000000000000000000000000000000000000000000000000000000000000000000000000000000090F4D3
:3DC8DF00020000000000000000000000000000000000000000000000000000000000000000000000000000000000000000000000000000000000000000000008ED25
:3DC91C00020000000000000000000000000000000000000000000000000000000000000000000000000000000000000000000000000000000000000000000008EDE7
:3DC95900000000000000000000000000000000000000000000000000000000000000000000000000000000000000000000000000000000000000000000000008EFAA
:3DC99600000000000000000000000000000000000000000000000000000000000000000000000000000000000000000000000000000000000000000000000080E7FD
:3DC9D300000000000000000000000000000000000000000000000000000000000000000000000000000000000000000000000000000000000000000000000080E7C0
:3DCA1000000000000000000000000000000000000000000000000000000000000000000000000000000000000000000000000000000000000000000000000080E782
:3DCA4D00000000000000000000000000000000000000000000000000000000000000000000000000000000000000000000000000000000000000000000000080E745
:3DCA8A000200000002000000000000000000000000000000000000000000000000000000000000004000000000000000000000000000000000000000000000088F94
:3DCAC7006280006000000000000000000000000000000000000000006010000000000000000000180000000000000000000000000000000000000000000000889D43
:3DCB0400020000000000000000000000000000000000000000000000000000000000000000000000000000000000000000000000000000000000000000000008EDFD
:3DCB4100420000400000000000000000000000000000000000000000400000000000000000000010000000000000000000000000000000000000000000000008BC21
:3DCB7E0080010080010000000000000000000000000000000000000080010000000000000000006000000000000000000000000000000000000000000000000098FF
:3DCBBB009E010080010000000000000000000000000000000000000080010000000000000000006000000000000000000000000000000000000000000000000086B6
:3DCBF8009E01008001000000000000000000000000000000000000008001000000000000000000600000000000000000000000000000000000000000000000888EE9
:3DCC35008001008001000000000000000000000000000000000000008001000000000000000000600000000000000000000000000000000000000000000000009847
:3DCC7200000110000110000110000110000110000110000110000110000110000000000040000440000440000440000440000440000440000440000440000480E721
:3DCCAF00000000000000000000000000000000000000000000000000000000000000000000000000000000000000000000000000000000000000000000000080E7E1
:3DCCEC00800118800118800118800118800118800118800118800118800118000000000060000660000660000660000660000660000660000660000660000680E7AD
:3DCD2900800008800008800008800008800008800008800008800008800008000000000020000220000220000220000220000220000220000220000220000280E76C
:3DCD660000005000000000000000000000000000000000000000000000001000000000000000200000000000000000000000000000000000000000000000008391FC
:3DCDA300000000000000000000000000000000000000000000000000000010000000000000000000000000000000000000000000000000000000000000000080F6CD
:3DCDE000000000000000000000000000000000000000000000000000000000000000000000000000000000000000000000000000000000000000000000000080E7AF
:3DCE1D00000000800000000000000000000000000000000000000000000000000000000000000020000000000000000000000000000000000000000000000000CD6B
:3DCE5A000000400000000000000000000000000000000000000000000000100000000000000020000000000000000000000000000000000000000000000000829019
:3DCE9700000000000000000000000000000000000000000000000000000000000000000000000000000000000000000000000000000000000000000000000080E7F7
:3DCED4000000000000000000000000000000000000000000000000000000000000000000000000000000000000000000000000000000000000000000000000E081C0
:3DCF11000020000000000000000000000000000000000000000000000000000000000000000400000000000000000000000000000000000000000000000000A0C35C
:3DCF4E00000000000000000000000000000000000000000000000000000008000000000000000000000000000000000000000000000000000000000000000012DEAE
:3DCF8B00000000400000000000000000000000000000000000000000000100000000000000000000000000000000000000000000000000000000000000100080A6F2
:3DCFC8000000000000000000000000000000000000000000000000000000000000000000000080004000000000000000000000000000000000000000000000C0EBC1
:3DD00500000000000000000000000000000000000000000000000000000000000000000000000000000000000000000000000000000000000000000000000080E787
:3DD04200000000000000000000000000000000000000000000000000000000000000000000000000000000000000000000000000000000000000000000000080E74A
:3DD07F00000000080000000000000000000000000000000000000000000000000000000000000000000000000000000000000000000000000000000000000080EFFD
:3DD0BC00000000000000000000000000000000000000000000000000000000000000000000000000000000000000000000000000000000000000000000000080E7D0
:3DD0F900000000000000000000000000000000000000000000000000000000000000000000000000000000000000000000000000000000000000000000000080E793
:3DD13600000000000000000000000000000000000000000000000000000000000000000000000000000000000000000000000000000000000000000000000080E755
:3DD17300000000000000000000000000000000000000000000000000000000000000000000000000000000000000000000000000000000000000000000000080E718
:3DD1B000000000000000000000000000000000000000000000000000000000000000000000000000000000000000000000000000000000000000000000000080E7DB
:3DD1ED00000000000000000000000000000000000000000000000000000000000000000000000000000000000000000000000000000000000000000000000080E79E
:3DD22A00000000000000000000000000000000000000000000000000000000000000000000000000000000000000000000000000000000000000000000000080E760
:3DD26700000000000000000000000000000000000000000000000000000000000000000000000000000000000000000000000000000000000000000000000080E723
:3DD2A400000000000000000000000000000000000000000000000000000000000000000000000000000000000000000000000000000000000000000000000080E7E6
:3DD2E100000000000000000000000000000000000000000000000000000000000000000000000000000000000000000000000000000000000000000000000080E7A9
:3DD31E00000000000000000000000000000000000000000000000000000000000000000000000000000000000000000000000000000000000000000000000080E76B
:3DD35B00000000000000000000000000000000000000000000000000000000000000000000000000000000000000000000000000000000000000000000000080E72E
:3DD39800000000000000000000000000000000000000000000000000000000000000000000000000000000000000000000000000000000000000000000000080E7F1
:3DD3D5000000000000000000000000000000000000000000000000000000000000000000000000000000000000000000000000000000000000000000000000A0C5B6
:3DD41200000000000000000000000000000000000000000000000000000000000000000000000000000000000000000000000000000000000000000000000008EFE6
:3DD44F00000000000000000000000000000000000000000000000000000000000000000000000000000000000000000000000000000000000000000000000080E739
:3DD48C00000000000000000000000000000000000000000000000000000000000000000000000000000000000000000000000000000000000000000000000080E7FC
:3DD4C900000000000000000000000000000000000000000000000000000000000000000000000000000000000000000000000000000000000000000000000080E7BF
:3DD50600000000000000000004000000000000000000000000000000000000000000000000000000000000000000000000000000000000000000000000000080A7BD
:3DD54300000000000000000000000000000000000000000000000000000000000000000000000000000000000000000000000000000000000000000000000080E744
:3DD58000000000000000000000000000000000000000000000000000000000000000000000000000000000000000000000000000000000000000000000000080E707
:3DD5BD00000000000000000000000000000000000000000000000000000000000000000000000000000000000000000000000000000000000000000000000080E7CA
:3DD5FA00000000000000000000000000000000000000000000000000000000000000000000000000000000000000000000000000000000000000000000000080E78D
:3DD63700000000000000000000000000000000000000000000000000000000000000000000000000000000000000000000000000000000000000000000000090F630
:3DD67400000000000000000000000000000000000000000000000000000000000000000000000000000000000000000000000000000000000000000000000080E712
:3DD6B100000000000000000000000000000000000000000000000000000000000000000000000000000000000000000000000000000000000000000000000080E7D5
:3DD6EE00000000000000000000000000000000000000000000000000000000000000000000000000000000000000000000000000000000000000000000000080E798
:3DD72B00000000000000000000000000000000000000000000000000000000000000000000000000000000000000000000000000000000000000000000000080E75A
:3DD76800000000000000000000000000000000000000000000000000000000000000000000000000000000000000000000000000000000000000000000000080E71D
:3DD7A5000000000000000000000000000000000000000000000000000000000000000000000000000000000000000000000000000000000000000000000000C0A3E4
:3DD7E200000000000000000000000000000000000000000000000000000000000000000000000000000000000000000000000000000000000000000000000080E7A3
:3DD81F00000000000000000000000000000000000000000000000000000000000000000000000000000000000000000000000000000000000000000000000080E765
:3DD85C00000000000000000000000000000000000000000000000000000000000000000000000000000000000000000000000000000000000000000000000080E728
:3DD89900000000000000000000000040000000000000000000000000000000000000000000000000000000000000000000000000000000000000000000000058FEBC
:3DD8D600000000000000000000000000000000000000000000000000000000000000000000000000000000000000000000000000000000000000000000000080E7AE
:3DD91300000000000000000040000000000000000000000000000000000000000000000000000000000000800002002000000000000000000000000000000000896C
:3DD95000000000000000000000000000000000000000000000000000000000000000000000000000000000000000000000000000000000000000000000000080E733
:3DD98D00000000000000000000000000000000000000000000000000000000000000000000000000000000000000000000000000000000000000000000000080E7F6
:3DD9CA00000000000000000000000000000000000000000000000000000000000000000000000000000000000000000000000000000000000000000000000008EF29
:3DDA07000000000000000000500000000000000000000000000000000000000000000000000000000000008000030020000000000000000000000000000000008867
:3DDA4400000110000110000110000110000110000110000110000110000110000000000040000440000440000440000440000440000440000440000440000480E741
:3DDA8100000000000000000000000000000000000000000000000000000000000000000000000000000000000000000000000000000000000000000000000080E701
:3DDABE00800118800118800118800118800118800118800118800118800118000000000060000660000660000660000660000660000660000660000660000608EF3D
:3DDAFB00820008800008800008800008800008800008800008800008800008000000000020000220000220000220000220000220000220000220000220000208EDFD
:3DDB3800020000000000000000000000000000000000000000000000000000000000000000000000000000000000000000000000000000000000000000000090F42A
:3DDB7500020000000000000000000000000000000000000000000000000000000000000000000000000000000000000000000000000000000000000000000008ED7C
:3DDBB200020000000000000000000000000000000000000000000000000000000000000000000000000000000000000000000000000000000000000000000008ED3F
:3DDBEF00000000000000000000000000000000000000000000000000000000000000000000000000000000000000000000000000000000000000000000000008EF02
:3DDC2C00000000000000000000000000000000000000000000000000000000000000000000000000000000000000000000000000000000000000000000000080E754
:3DDC6900000000000000000000000000000000000000000000000000000000000000000000000000000000000000000000000000000000000000000000000080E717
:3DDCA600000000000000000000000000000000000000000000000000000000000000000000000000000000000000000000000000000000000000000000000080E7DA
:3DDCE300000000000000000000000000000000000000000000000000000000000000000000000000000000000000000000000000000000000000000000000008EF0D
:3DDD2000020000000000000000000000000000000000000000000000000000000000000000000000000080000000000002000000000000000000000000000088CDED
:3DDD5D00020000000000000000000000000000000000000000000000000000000000000000000000000018000000800100000000000000000000000000000090F46A
:3DDD9A00020000000000000000000000000000000000000000000000000000000000000000000000000000000000000000000000000000000000000000000008ED55
:3DDDD700020000000000000000000000000000000000000000000000000000000000000000000000000010000000000100000000000000000000000000000008ED07
:3DDE1400000000000000000000000000000000000000000000000000000000000000000000000000000060000000000600000000000000000000000000000008EF74
:3DDE5100000000000000000000000000000000000000000000000000000000000000000000000000000060000000000600000000000000000000000000000080E7C7
:3DDE8E00000000000000000000000000000000000000000000000000000000000000000000000000000060000000000600000000000000000000000000000008EFFA
:3DDECB00020000000000000000000000000000000000000000000000000000000000000000000000000060000000000600000000000000000000000000000008EDBD
:3DDF0800020000000000000000000000000000000000000000000000000000000000000000000000000000000000000000000000000000000000000000000090F456
:3DDF4500020000000000000000000000000000000000000000000000000000000000000000000000000000000000000000000000000000000000000000000008EDA8
:3DDF8200020000000000000000000000000000000000000000000000000000000000000000000000000000000000000000000000000000000000000000000008ED6B
:3DDFBF00000000000000000000000000000000000000000000000000000000000000000000000000000000000000000000000000000000000000000000000008EF2E
:3DDFFC00000000000000000000000000000000000000000000000000000000000000000000000000000000000000000000000000000000000000000000000080E781
:3DE03900000000000000000000000000000000000000000000000000000000000000000000000000000000000000000000000000000000000000000000000080E743
:3DE07600000000000000000000000000000000000000000000000000000000000000000000000000000000000000000000000000000000000000000000000080E706
:3DE0B300000000000000000000000000000000000000000000000000000000000000000000000000000000000000000000000000000000000000000000000008EF39
:3DE0F000020000000000001000000000000000000000000000000000000000000000000000000000000000000004000000000000000000000000000000000008AC29
:3DE12D00020000000000600200000000000000000000000000000000000000000000000000000000000000800100000000000000000000000000000000000010AF11
:3DE16A00020000000000000000000000000000000000000000000000000000000000000000000000000000000000000000000000000000000000000000000008ED81
:3DE1A700020000000000400000000000000000000000000000000000000000000000000000000000000000000100000000000000000000000000000000000008BC34
:3DE1E400000000000000800100000000000000000000000000000000000000000000000000000000000000000600000000000000000000000000000000000088905F
:3DE2210000000000000080010000000000000000000000000000000000000000000000000000000000000000060000000000000000000000000000000000000098A1
:3DE25E0000000000000080010000000000000000000000000000000000000000000000000000000000000000060000000000000000000000000000000000008890E4
:3DE29B0002000000000080010000000000000000000000000000000000000000000000000000000000000000060000000000000000000000000000000000008892A3
:3DE2D800020000000000000000000000000000000000000000000000000000000000000000000000000000000000000000000000000000000000000000000090F483
:3DE31500020000000000000000000000000000000000000000000000000000000000000000000000000000000000000000000000000000000000000000000008EDD4
:3DE35200020000000000000000000000000000000000000000000000000000000000000000000000000000000000000000000000000000000000000000000008ED97
:3DE38F00000000000000000000000000000000000000000000000000000000000000000000000000000000000000000000000000000000000000000000000008EF5A
:3DE3CC00000000000000000000000000000000000000000000000000000000000000000000000000000000000000000000000000000000000000000000000080E7AD
:3DE40900000000000000000000000000000000000000000000000000000000000000000000000000000000000000000000000000000000000000000000000080E76F
:3DE44600000000000000000000000000000000000000000000000000000000000000000000000000000000000000000000000000000000000000000000000080E732
:3DE48300000000000000000000000000000000000000000000000000000000000000000000000000000000000000000000000000000000000000000000000008EF65
:3DE4C000020000000000000000000000000000000000000000000000000000000000000000000000000000000000000000000000000000000000000000000008ED28
:3DE4FD000200000000000000000000000000000000000000000000000000000000000000000000008009040000182000000000000000000000000000000000109477
:3DE53A00020000000000000000000000000000000000000000000000000000000000000000000000000000000000000000000000000000000000000000000008EDAD
:3DE57700020000000000000000000000000000000000000000000000000000000000000000000000000100000010000000000000000000000000000000000008ED5F
:3DE5B400000000000000000000000000000000000000000000000000000000000000000000000000000600000060000000000000000000000000000000000008EFCD
:3DE5F100000000000000000000000000000000000000000000000000000000000000000000000000000600000060000000000000000000000000000000000080E720
:3DE62E00000000000000000000000000000000000000000000000000000000000000000000000000000600000060000000000000000000000000000000000008EF52
:3DE66B00020000000000000000000000000000000000000000000000000000000000000000000000000600000060000000000000000000000000000000000008ED15
:3DE6A800020000000000000020000000000000000000000000000000000000000000000000000000000000000000000000000000000000000000000000000090D6AD
:3DE6E500020000000000000026000000000000000000000000000000000000000000000000000000000000000000000000000000000000000000000000000008AF19
:3DE72200020000000000000000000000000000000000000000000000000000000000000000000000000000000000000000000000000000000000000000000008EDC3
:3DE75F00000000000000000004000000000000000000000000000000000000000000000000000000000000000000000000000000000000000000000000000008AFC2
:3DE79C00000000000000000018000000000000000000000000000000000000000000000000000000000000000000000000000000000000000000000000000000FE2A
:3DE7D900000000000000000018000000000000000000000000000000000000000000000000000000000000000000000000000000000000000000000000000000FEED
:3DE81600000000000000000018000000000000000000000000000000000000000000000000000000000000000000000000000000000000000000000000000000FEAF
:3DE85300000000000000000018000000000000000000000000000000000000000000000000000000000000000000000000000000000000000000000000000000FE72
:3DE89000020000000000000000000001000000000000000000000000000000000000000000000000000000000000000000000000000000000000000000000008FD43
:3DE8CD000200000000060100006002260200000000000000000000000000000000000000000000000000000000000000000000000000000000000000000000088EE5
:3DE90A00020000000000000000000000000000000000000000000000000000000000000000000000000000000000000000000000000000000000000000000008EDD9
:3DE94700020000000004000000400004000000000000000000000000000000000000000000000000000000000000000000000000000000000000000000000008AD94
:3DE98400000000000018000000800118000000000000000000000000000000000000000000000000000000000000000000000000000000000000000000000000FEA7
:3DE9C1001E0000000018000000800118000000000000000000000000000000000000000000000000000000000000000000000000000000000000000000000000E06A
:3DE9FE001E0000000018000000800118000000000000000000000000000000000000000000000000000000000000000000000000000000000000000000000000E02D
:3DEA3B00000000000018000000800118000000000000000000000000000000000000000000000000000000000000000000000000000000000000000000000000FEEF
:3DEA7800000110000110000110000110000110000110000110000110000110000000000040000440000440000440000440000440000440000440000440000480E7FD
:3DEAB500000000000000000000000000000000000000000000000000000000000000000000000000000000000000000000000000000000000000000000000080E7BD
:3DEAF200800118800118800118800118800118800118800118800118800118000000000060000660000660000660000660000660000660000660000660000680E789
:3DEB2F00800008800008800008800008800008800008800008800008800008000000000020000220000220000220000220000220000220000220000220000280E748
:3DEB6C0000000000000000004000000000000000000000000000000000000000000000000000000000200000000000000300000000000000000000000000008091F8
:3DEBA900000000000000000000000000000000000000000000000000000000000000000000000000000000000000000000000000000000000000000000000080E7C8
:3DEBE600000000000000000000000000000000000000000000000000000000000000000000000000000000000000000000000000000000000000000000000080E78B
:3DEC2300000000000008000000800008000000000000000000000000000000000000000000000000000000000000000000000000000000000000000000000000EF35
:3DEC60000000000000000000400000000000000000000000000000000000000000000000000000000020000000000000020000000000000000000000000000808114
:3DEC9D00000000000000000000000000000000000000000000000000000000000000000000000000000000000000000000000000000000000000000000000080E7D3
:3DECDA000000000000000000000000000000000000000000000000000000000000000000000000000000000000000000000000000000000000000000000000E0819C
:3DED1700000000000000000000000000000000000000000000000000000000000000000000000000000000000000080000000000000000000000000000000080EF48
:3DED5400000000000000800000008000000000000000000000000000000000000000000000000000000000000000000000000000000000000000000000000000E79B
:3DED9100000000000010000000000000000000000000000000000000000000000000000000000000000010000000000000000000000000000000000000000080E7BE
:3DEDCE000000000000000000000000000000000000000000000000000000000000000000000000000000000000040080000000000000000000000000000000C0EBD9
:3DEE0B00000000000000000000000000000000000000000000000000000000000000000000000000000000000000000000000000000000000000000000000080E763
:3DEE4800000000000000000000000000000000000000000000000000000000000000000000000000000000000000000000000000000000000000000000000080E726
:3DEE8500000000000000000000000000000000000000000000000000000000000000000000000000000002000000000000000000000000000000000000000080C707
:3DEEC200000000000000000000000000000000000000000000000000000000000000000000000000000000000000000000000000000000000000000000000080E7AC
:3DEEFF000000000000000000000000000000000000000000000000000000000000000000000000000000000000000000000000000000000000000000000000B0D452
:3DEF3C00000000000000000000000000000000000000000000000000000000000000000000000000000000000000000000000000000000000000000000000080E731
:3DEF7900000000000000000000000000000000000000000000000000000000000000000000000000000000000000000000000000000000000000000000000080E7F4
:3DEFB600000000000000000000000000000000000000000000000000000000000000000000000000000000000000000000000000000000000000000000000080E7B7
:3DEFF300000000000000000000000000000000000000000000000000000000000000000000000000000000000000000000000000000000000000000000000080E77A
:3DF03000000000000000000000000000000000000000000000000000000000000000000000000000000000000000000000000000000000000000000000000080E73C
:3DF06D00000000000000000000000000000000000000000000000000000000000000000000000000000000000000000000000000000000000000000000000080E7FF
:3DF0AA00000000000000000000000000000000000000000000000000000000000000000000000000000000000000000000000000000000000000000000000080E7C2
:3DF0E700000000000000000000000000000000000000000000000000000000000000000000000000000000000000000000000000000000000000000000000080E785
:3DF12400000000000000000000000000000000000000000000000000000000000000000000000000000000000000000000000000000000000000000000000080E747
:3DF16100000000000000000000000000000000000000000000000000000000000000000000000000000000000000000000000000000000000000000000000080E70A
:3DF19E00000000000000000000000000000000000000000000000000000000000000000000000000000000000000000000000000000000000000000000000080E7CD
:3DF1DB00000000000000000000000000000000000000000000000000000000000000000000000000000000000000000000000000000000000000000000000080E790
:3DF21800000000000000000000000000000000000000000000000000000000000000000000000000000000000000000000000000000000000000000000000080E752
:3DF25500000000000000000000000000000000000000000000000000000000000000000000000000000000000000000000000000000000000000000000000080E715
:3DF29200000000000000000000000000000000000000000000000000000000000000000000000000000000000000000000000000000000000000000000000080E7D8
:3DF2CF00000000000000000000000000000000000000000000000000000000000000000000000000000000000000000000000000000000000000000000000080E79B
:3DF30C000000000000000000000000000000000000000000000000000000000000000000000000000000000000000000000000000000000000000000000000A0C55F
:3DF34900000000000000000000000000000000000000000000000000000000000000000000000000000000000000000000000000000000000000000000000090F601
:3DF38600000000000000000000000000000000000000000000000000000000000000000000000000000000000000000000000000000000000000000000000080E7E3
:3DF3C300000000000000000000000000000000000000000000000000000000000000000000000000000000000000000000000000000000000000000000000080E7A6
:3DF40000000000000000000000000000000000000000000000000000000000000000000000000000000000000000000000000000000000000000000000000080E768
:3DF43D00000000000000000000000000000000000000000000000000000000000000000000000000000000000000000000000000000000000000000000000080E72B
:3DF47A00000000000000000000000000000000000000000000000000000000000000000000000000000000000000000000000000000000000000000000000008EF5E
:3DF4B700000000000000000000000000000000000000000000000000000000000000000000000000000000000000000000000000000000000000000000000080E7B1
:3DF4F4000000000000000000000000000000000000000000000000000000000000000000000000000000000000000000000000000000000000000000000000C0A378
:3DF53100000000000000000000000000000000000000000000000000000000000000000000000000000000000000000000000000000000000000000000000080E736
:3DF56E00000000000000000000000000000000000000000000000000000000000000000000000000000000000000000000000000000000000000000000000080E7F9
:3DF5AB00000000000000000000000000000000000000000000000000000000000000000000000000000000000000000000000000000000000000000000000080E7BC
:3DF5E800000000000000000000000000000000000000000000000000000000000000000000000000000000000000000000000000000000000000000000000080E77F
:3DF62500000000000000000000000000000000000000000000000000000000000000000000000000000000000000000000000000000000000000000000000080E741
:3DF66200000000000000000000000000000000000000000000000000000000000000000000000000000000000000000000000000000000000000000000000080E704
:3DF69F00000000000000000000000000000000000000000000000000000000000000000000000000000000000000000000000000000000000000000000000038DC1A
:3DF6DC00000000000000000000000000000000000000000000000000000000000000000000000000000000000000000000000000000000000000000000000080E78A
:3DF71900000000000000000000000000000000010000000000000000000000000000000000000000000000000000000000000002800800000000000000000080CEDA
:3DF75600000000000000000000000000000000000000000000000000000000000000000000000000000000000000000000000000000000000000000000000080E70F
:3DF79300000000000000000000000000000000000000000000000000000000000000000000000000000000000000000000000000000000000000000000000080E7D2
:3DF7D000000000000000000000000000000000000000000000000000000000000000000000000000000000000000000000000000000000000000000000000080E795
:3DF80D00000000000000000000000000000000010000000000000000000000000000000000000000000000000000000000000002800C000000000000000000808A25
:3DF84A00000110000110000110000110000110000110000110000110000110000000000040000440000440000440000440000440000440000440000440000480E71D
:3DF88700000000000000000000000000000000000000000000000000000000000000000000000000000000000000000000000000000000000000000000000080E7DD
:3DF8C400800118800118800118800118800118800118800118800118800118000000000060000660000660000660000660000660000660000660000660000608EF19
:3DF90100820008800008800008800008800008800008800008800008800008000000000020000220000220000220000220000220000220000220000220000208EDD8
:3DF93E00020000000000000000000000000000000000000000000000000000000000000000000000000000000000000000000000000000000000000000000090F406
:3DF97B00020000000000000000000000000000000000000000000000000000000000000000000000000000000000000000804100000000000000000000000088F014
:3DF9B800020000000000000000000000000000000000000000000000000000000000000000000000000000000000000000000000000000000000000000000008ED1B
:3DF9F500000000000000000000000000000000000000000000000000000000000000000000000000000000000000000000000100000000000000000000000008FECE
:3DFA32000000000000000000000000000000000000000000000000000000000000000000000000000000000000000000000006000000000000000000000000808190
:3DFA6F000000000000000000000000000000000000000000000000000000000000000000000000000000000000000000000006000000000000000000000000808153
:3DFAAC000000000000000000000000000000000000000000000000000000000000000000000000000000000000000000000006000000000000000000000000808116
:3DFAE9000000000000000000000000000000000000000000000000000000000000000000000000000000000000000000000006000000000000000000000000088949
:3DFB2600020000000000000000000000000000000000000000000000000000000000000000000000000000000000000000000000000000000000000000000008EDAB
:3DFB63000200000000000000000000000000060800000000000000000000000000000000000000000000000000000000000000000000000000000000000000909C29
:3DFBA000020000000000000000000000000000000000000000000000000000000000000000000000000000000000000000000000000000000000000000000008ED31
:3DFBDD00020000000000000000000000000004000000000000000000000000000000000000000000000000000000000000000000000000000000000000000008AD30
:3DFC1A00000000000000000000000000000018000000000000000000000000000000000000000000000000000000000000000000000000000000000000000088F617
:3DFC5700000000000000000000000000000018000000000000000000000000000000000000000000000000000000000000000000000000000000000000000000FE5A
:3DFC9400000000000000000000000000000018000000000000000000000000000000000000000000000000000000000000000000000000000000000000000088F69D
:3DFCD100020000000000000000000000000018000000000000000000000000000000000000000000000000000000000000000000000000000000000000000088F460
:3DFD0E00020000000000000000000000000000000000000000000000000000000000000000000000000000000000000000000000000000000000000000000090F432
:3DFD4B00020000000000000000000000000000000000000000000000000000000000000000000000000000000000000000000000000000000000000000000008ED84
:3DFD8800020000000000000000000000000000000000000000000000000000000000000000000000000000000000000000000000000000000000000000000008ED47
:3DFDC500000000000000000000000000000000000000000000000000000000000000000000000000000000000000000000000000000000000000000000000008EF0A
:3DFE0200000000000000000000000000000000000000000000000000000000000000000000000000000000000000000000000000000000000000000000000080E75C
:3DFE3F00000000000000000000000000000000000000000000000000000000000000000000000000000000000000000000000000000000000000000000000080E71F
:3DFE7C00000000000000000000000000000000000000000000000000000000000000000000000000000000000000000000000000000000000000000000000080E7E2
:3DFEB900000000000000000000000000000000000000000000000000000000000000000000000000000000000000000000000000000000000000000000000008EF15
:3DFEF600020000000000000000000000000000000000000000000000000000000000000000000000000000000000000000000000000002000000000000000008CDF6
:3DFF3300020000000000000000000000000000000000000000000000000000000000000000000000000000000000000000000098A00100000000000000000010D472
:3DFF7000020000000000000000000000000000000000000000000000000000000000000000000000000000000000000000000000000000000000000000000008ED5D
:3DFFAD00020000000000000000000000000000000000000000000000000000000000000000000000000000000000000000000010000100000000000000000008ED0F
:16FFEA00FFFFFFFFFFFFFFFFFFFFFFFFFFFFFFFFFFFFFFFFFFFF17
:020000040001F9
:3D000000000000000000000000000000000000000000000000000000000000000000000000000000000000000000000000000060000600000000000000000008EF66
:3D003D00000000000000000000000000000000000000000000000000000000000000000000000000000000000000000000000060000600000000000000000080E7B9
:3D007A00000000000000000000000000000000000000000000000000000000000000000000000000000000000000000000000060000600000000000000000008EFEC
:3D00B700020000000000000000000000000000000000000000000000000000000000000000000000000000000000000000000060000600000000000000000008EDAF
:3D00F400020000000000000000000000000000000000000000000000000000000000000000000000000000000000000000000000000000000000000000000090F449
:3D013100020000000000000000000000000000000000000000000000000000000000000000000000000000000000000000000000000000000000000000000008ED9A
:3D016E00020000000000000000000000000000000000000000000000000000000000000000000000000000000000000000000000000000000000000000000008ED5D
:3D01AB00000000000000000000000000000000000000000000000000000000000000000000000000000000000000000000000000000000000000000000000008EF20
:3D01E800000000000000000000000000000000000000000000000000000000000000000000000000000000000000000000000000000000000000000000000080E773
:3D022500000000000000000000000000000000000000000000000000000000000000000000000000000000000000000000000000000000000000000000000080E735
:3D026200000000000000000000000000000000000000000000000000000000000000000000000000000000000000000000000000000000000000000000000080E7F8
:3D029F00000000000000000000000000000000000000000000000000000000000000000000000000000000000000000000000000000000000000000000000008EF2B
:3D02DC00020000000000000000000000000000000200000000000000000000000000000000000000000000000000000000000000000000000000000000000008CF0A
:3D031900020000000000000000000000000000600200000000000000000000000000000000000000000000000000000000000000000000000000000000000090B6FD
:3D035600020000000000000000000000000000000000000000000000000000000000000000000000000000000000000000000000000000000000000000000008ED73
:3D039300020000000000000000000000000000400000000000000000000000000000000000000000000000000000000000000000000000000000000000000008AD36
:3D03D000000000000000000000000000000000800100000000000000000000000000000000000000000000000000000000000000000000000000000000000088F6F1
:3D040D00000000000000000000000000000000800100000000000000000000000000000000000000000000000000000000000000000000000000000000000000FE33
:3D044A00000000000000000000000000000000800100000000000000000000000000000000000000000000000000000000000000000000000000000000000000FEF6
:3D048700020000000000000000000000000000800100000000000000000000000000000000000000000000000000000000000000000000000000000000000088F439
:3D04C400020000000000000000000000000000000000000000000000000000000000000000000000000000000000000000000000000000000000000000000008ED04
:3D050100020000000000000000000000000000000000000000000000000000000000000000000000000000000000000098400000000000000000000000000008B427
:3D053E00020000000000000000000000000000000000000000000000000000000000000000000000000000000000000000000000000000000000000000000008ED89
:3D057B00000000000000000000000000000000000000000000000000000000000000000000000000000000000000000010000000000000000000000000000080F6BD
:3D05B80000000000000000000000000000000000000000000000000000000000000000000000000000000000000000006000000000000000000000000000008081A5
:3D05F5000000000000000000000000000000000000000000000000000000000000000000000000000000000000000000600000000000000000000000000000808168
:3D063200000000000000000000000000000000000000000000000000000000000000000000000000000000000000000060000000000000000000000000000080812A
:3D066F0000000000000000000000000000000000000000000000000000000000000000000000000000000000000000006000000000000000000000000000008081ED
:3D06AC00020000000000000000000000000001000000100200000000000000000000000000000000000000000000000000000000000000040000000000000008CB25
:3D06E900020000000000000000000000600000000026600000000000000000000000000000000000000000000000000000000000000098000000000000000008B696
:3D072600020000000000000000000000000000000000000000000000000000000000000000000000000000000000000000000000000000000000000000000008ED9F
:3D076300020000000000000000000000400000000004400000000000000000000000000000000000000000000000000000000000000010000000000000000008BCFF
:3D07A000000000000000000000000000800100000018800100000000000000000000000000000000000000000000000000000000000060000000000000000000980A
:3D07DD001E000000000000000000000080010000001880010000000000000000000000000000000000000000000000000000000000006000000000000000000086C1
:3D081A001E00000000000000000000008001000000188001000000000000000000000000000000000000000000000000000000000000600000000000000000989FD2
:3D0857000000000000000000000000008001000000188001000000000000000000000000000000000000000000000000000000000000600000000000000000009852
:3D089400000110000110000110000110000110000110000110000110000110000000000040000440000440000440000440000440000440000440000440000480E7C3
:3D08D100000000000000000000000000000000000000000000000000000000000000000000000000000000000000000000000000000000000000000000000080E783
:3D090E00800118800118800118800118800118800118800118800118800118000000000060000660000660000660000660000660000660000660000660000680E74E
:3D094B00800008800008800008800008800008800008800008800008800008000000000020000220000220000220000220000220000220000220000220000280E70E
:3D09880000000000000000000000000000000000000014000000000000000000000000000000000000000000000000000000A000000000000000000000000080F905
:3D09C500000000000000000000000000000000000000000000000000000000000000000000000000000000000000000000000000000000000000000000000080E78E
:3D0A0200000000000000000000000000000000000000000000000000000000000000000000000000000000000000000000000000000000000000000000000080E750
:3D0A3F00000000000000000000000000800000000000800000000000000000000000000000000000000000000000000000000000000020000000000000000080C515
:3D0A7C00000000000000000000000000000000000008100000000000000000000000000000000000000000000000000000002000000000000000000000000000FD08
:3D0AB900000000000000000000000000000000000000000000000000000000000000000000000000000000000000000000000000000000000000000000000080E799
:3D0AF6000000000000000000000000000000000000000000000000000000000000000000000000000000000000000000000000000000000000000000000000A0C55E
:3D0B3300000000000000000000000000000000020000000000000000000000000000000000000000000000000000000000000000000000000000000000000080E51E
:3D0B7000000000000000000000000000000000000000080000000000000000000000000000000000000000000000000000000000000020000000000000000080CDD3
:3D0BAD00000000000000000000000000000000000000400000000000000000000000000000000000000000000000000000000400100000000000000000000080F344
:3D0BEA00000000000000000000000000000001400000000000000000000000000000000000000000000000000000000000000000008000000000000000000080BFCE
:3D0C2700000000000000000000000000000000000000000000000000000000000000000000000000000000000000000000000000000000000000000000000080E729
:3D0C6400000000000000000000000000000000000000000000000000000000000000000000000000000000000000000000000000000000000000000000000080E7EC
:3D0CA100000000000000000000000000000000000000000000000000000000000000000000000000000000000000000000200000000000000000000000000080C7AF
:3D0CDE00000000000000000000000000000000000000000000000000000000000000000000000000000000000000000000000000000000000000000000000080E772
:3D0D1B00000000000000000000000000000000000000000000000000000000000000000000000000000000000000000000000000000000000000000000000080E734
:3D0D58000000000000000000000000000000000000000000000000000000000000000000000000000000000000000000000000000000000000000000000000C0A3FB
:3D0D9500000000000000000000000000000000000000000000000000000000000000000000000000000000000000000000000000000000000000000000000080E7BA
:3D0DD200000000000000000000000000000000000000000000000000000000000000000000000000000000000000000000000000000000000000000000000080E77D
:3D0E0F00000000000000000000000000000000000000000000000000000000000000000000000000000000000000000000000000000000000000000000000080E73F
:3D0E4C000000000000000000000000000000000000000000000000000000000000000000000000000000000000000000000000000000000000000000000000A0C504
:3D0E8900000000000000000000000000000000000000000000000000000000000000000000000000000000000000000000000000000000000000000000000080E7C5
:3D0EC600000000000000000000000000000000000000000000000000000000000000000000000000000000000000000000000000000000000000000000000080E788
:3D0F0300000000000000000000000000000000000000000000000000000000000000000000000000000000000000000000000000000000000000000000000080E74A
:3D0F4000000000000000000000000000000000000000000000000000000000000000000000000000000000000000000000000000000000000000000000000080E70D
:3D0F7D00000000000000000000000000000000000000000000000000000000000000000000000000000000000000000000000000000000000000000000000080E7D0
:3D0FBA00000000000000000000000000000000000000000000000000000000000000000000000000000000000000000000000000000000000000000000000080E793
:3D0FF700000000000000000000000000000000000000000000000000000000000000000000000000000000000000000000000000000000000000000000000080E756
:3D103400000000000000000000000000000000000000000000000000000000000000000000000000000000000000000000000000000000000000000000000080E718
:3D107100000000000000000000000000000000000000000000000000000000000000000000000000000000000000000000000000000000000000000000000080E7DB
:3D10AE00000000000000000000000000000000000000000000000000000000000000000000000000000000000000000000000000000000000000000000000080E79E
:3D10EB00000000000000000000000000000000000000000000000000000000000000000000000000000000000000000000000000000000000000000000000090F642
:3D112800000000000000000000000000000000000000000000000000000000000000000000000000000000000000000000000000000000000000000000000080E723
:3D1165000000000000000000000000000000000000000000000000000000000000000000000000000000000000000000000000000000000000000000000000C0A3EA
:3D11A200000000000000000000000000000000000000000000000040000000000000000000000000000000000000000000000000000000000000000000000080A3AD
:3D11DF00000000000000000000000000000000000000000000000000000000000000000000000000000000000000000000000000000000000000000000000080E76C
:3D121C00000000000000000000000000000000000000000000000000000000000000000000000000000000000000000000000000000000000000000000000080E72E
:3D125900000000000000000000000000000000000000000000000000000000000000000000000000000000000000000000000000000000000000000000000028CD63
:3D129600000000000000000000000000000000000000000000000000000000000000000000000000000000000000000000000000000000000000000000000080E7B4
:3D12D300000000000000000000000000000000000000000000000000000000000000000000000000000000000000000000000000000000000000000000000080E777
:3D131000000000000000000000000000000000000000000000000000000000000000000000000000000000000000000000000000000000000000000000000080E739
:3D134D00000000000000000000000000000000000000000000000000000000000000000000000000000000000000000000000000000000000000000000000080E7FC
:3D138A00000000000000000000000000000000000000000000000000000000000000000000000000000000000000000000000000000000000000000000000080E7BF
:3D13C700000000000000000000000000000000000000000000000000000000000000000000000000000000000000000000000000000000000000000000000080E782
:3D140400000000000000000000000000000000000000000000000000000000000000000000000000000000000000000000000000000000000000000000000080E744
:3D144100000000000000000000000000000000000000000000000000000000000000000000000000000000000000000000000000000000000000000000000080E707
:3D147E00000000000000000000000000000000000000000000000000000000000000000000000000000000000000000000000000000000000000000000000080E7CA
:3D14BB000000000000000000000000000000000000000000000000000000000000000000000000000000000000000000000000000000000000000000000000A0C58F
:3D14F800000000000000000000000000000000000000000000000000000000000000000000000000000000000000000000000000000000000000000000000080E750
:3D153500000000000000000000000000000000000000000000100040000000010000000000000000000000000000000000000000000000000008000000000000BA66
:3D157200000000000000000000000000000000000000000000000000000000000000000000000000000000000000000000000000000000000000000000000080E7D5
:3D15AF00100000000000000000000000000000000000000000000000000000000000000000000000000000000000000000000000000000000000000000000080F778
:3D15EC00000000000000000000000000000000000000000000000000000000000000000000000000000000000000000000000000000000000000000000000080E75B
:3D162900000000000000000000000000000000000000000000100050000000010000000000000000000000000000000000000000000000000008000000000000AB70
:3D166600000110000110000110000110000110000110000110000110000110000000000040000440000440000440000440000440000440000440000440000480E7E3
:3D16A300000000000000000000000000000000000000000000000000000000000000000000000000000000000000000000000000000000000000000000000080E7A3
:3D16E000800118800118800118800118800118800118800118800118800118000000000060000660000660000660000660000660000660000660000660000608EFDF
:3D171D00820008800008800008800008800008800008800008800008800008000000000020000220000220000220000220000220000220000220000220000208ED9E
:3D175A00020000000000000000000000000000000000000000000000000000000000000000000000000000000000000000000000000000000000000000000090F4CC
:3D1797000200000000000000000000000000000000000000060100000000000000000000000000000000000000000000000000000000000000000000000000088C78
:3D17D400020000000000000000000000000000000000000000000000000000000000000000000000000000000000000000000000000000000000000000000008EDE1
:3D181100000000000000000000000000000000000000000004000000000000000000000000000000000000000000000000000000000000000000000000000008AFDF
:3D184E00000000000000000000000000000000000000000018000000000000000000000000000000000000000000000000000000000000000000000000000000FE47
:3D188B00000000000000000000000000000000000000000018000000000000000000000000000000000000000000000000000000000000000000000000000000FE0A
:3D18C800000000000000000000000000000000000000000018000000000000000000000000000000000000000000000000000000000000000000000000000000FECD
:3D190500000000000000000000000000000000000000000018000000000000000000000000000000000000000000000000000000000000000000000000000088F60F
:3D194200020000000000000000000000000000000000000000000000000000100000000000000000000000000000000000000000000000000000000000000008FD51
:3D197F0002000000000000000000000000000000000000000000000000000600000000000000000000000000000000000000000000000000000000000000009094FF
:3D19BC00020000000000000000000000000000000000000000000000000000000000000000000000000000000000000000000000000000000000000000000008EDF7
:3D19F900020000000000000000000000000000000000000000000000000004000000000000000000000000000000000000000000000000000000000000000008ADF6
:3D1A3600000000000000000000000000000000000000000000000000000018000000000000000000000000000000000000000000000000000000000000000088F6DD
:3D1A7300000000000000000000000000000000000000000000000000000018000000000000000000000000000000000000000000000000000000000000000000FE20
:3D1AB000000000000000000000000000000000000000000000000000000018000000000000000000000000000000000000000000000000000000000000000088F663
:3D1AED00020000000000000000000000000000000000000000000000000018000000000000000000000000000000000000000000000000000000000000000088F426
:3D1B2A00020000000000000000000000000000000000000000000000000000000000000000000000000000000000000000000000000000000000000000000090F4F8
:3D1B6700020000000000000000000000000000000000000000000000000000000000000000000000000000000000000000000000000000000000000000000008ED4A
:3D1BA400020000000000000000000000000000000000000000000000000000000000000000000000000000000000000000000000000000000000000000000008ED0D
:3D1BE100000000000000000000000000000000000000000000000000000000000000000000000000000000000000000000000000000000000000000000000008EFD0
:3D1C1E00000000000000000000000000000000000000000000000000000000000000000000000000000000000000000000000000000000000000000000000080E722
:3D1C5B00000000000000000000000000000000000000000000000000000000000000000000000000000000000000000000000000000000000000000000000080E7E5
:3D1C9800000000000000000000000000000000000000000000000000000000000000000000000000000000000000000000000000000000000000000000000080E7A8
:3D1CD500000000000000000000000000000000000000000000000000000000000000000000000000000000000000000000000000000000000000000000000008EFDB
:3D1D1200020000000000000000000000000000000000000000000000000000000000000000000000000000000000000000000000000000000000000000000008ED9D
:3D1D4F00020000000000000000000000000000000000000000608000000000000000000000000000000000000000000000000000000000000098200000000090A588
:3D1D8C00020000000000000000000000000000000000000000000000000000000000000000000000000000000000000000000000000000000000000000000008ED23
:3D1DC900020000000000000000000000000000000000000000400000000000000000000000000000000000000000000000000000000000000010000000000008BCC7
:3D1E060000000000000000000000000000000000000000000080010000000000000000000000000000000000000000000000000000000000006000000000008890A6
:3D1E430000000000000000000000000000000000000000000080010000000000000000000000000000000000000000000000000000000000006000000000000098E9
:3D1E8000000000000000000000000000000000000000000000800100000000000000000000000000000000000000000000000000000000000060000000000088902C
:3D1EBD0002000000000000000000000000000000000000000080010000000000000000000000000000000000000000000000000000000000006000000000008892EB
:3D1EFA00020000000000000000000000000000000000000000000000020000000000000000000000000000000000000000000000000000000000000000000090F621
:3D1F3700020000000000000000000000000000000000000000000026000000000000000000000000000000000000000000000000000000000000000000000008AF8E
:3D1F7400020000000000000000000000000000000000000000000000000000000000000000000000000000000000000000000000000000000000000000000008ED39
:3D1FB100000000000000000000000000000000000000000000000004000000000000000000000000000000000000000000000000000000000000000000000008AF38
:3D1FEE00000000000000000000000000000000000000000000000018000000000000000000000000000000000000000000000000000000000000000000000000FEA0
:3D202B00000000000000000000000000000000000000000000000018000000000000000000000000000000000000000000000000000000000000000000000000FE62
:3D206800000000000000000000000000000000000000000000000018000000000000000000000000000000000000000000000000000000000000000000000000FE25
:3D20A500000000000000000000000000000000000000000000000018000000000000000000000000000000000000000000000000000000000000000000000088F668
:3D20E200020000000000000000000000000000000000000000000000000000000000000000000000000000000000000000000000000000000000000004000008AD06
:3D211F00020000000000000000000000000000000000000000000000000000000000000000000000000000000000000000000000000000000000800900000090ED7B
:3D215C00020000000000000000000000000000000000000000000000000000000000000000000000000000000000000000000000000000000000000000000008ED4F
:3D219900020000000000000000000000000000000000000000000000000000000000000000000000000000000000000000000000000000000000000100000008FC02
:3D21D6000000000000000000000000000000000000000000000000000000000000000000000000000000000000000000000000000000000000000006000000088935
:3D2213000000000000000000000000000000000000000000000000000000000000000000000000000000000000000000000000000000000000000006000000808187
:3D22500000000000000000000000000000000000000000000000000000000000000000000000000000000000000000000000000000000000000000060000000889BA
:3D228D000200000000000000000000000000000000000000000000000000000000000000000000000000000000000000000000000000000000000006000000088B79
:3D22CA00020000000000000000000000000000000000000000000000000000000000000000000000000000000000000000000000000000000002000000000090D46F
:3D230700020000000000000000000000000000000000000000000000000000000000000000000000000000000000000000000000000000800100000000000088F49A
:3D234400020000000000000000000000000000000000000000000000000000000000000000000000000000000000000000000000000000000000000000000008ED65
:3D238100000000000000000000000000000000000000000000000000000000000000000000000000000000000000000000000000000000000100000000000008FE18
:3D23BE0000000000000000000000000000000000000000000000000000000000000000000000000000000000000000000000000000000000060000000000008081DB
:3D23FB00000000000000000000000000000000000000000000000000000000000000000000000000000000000000000000000000000000000600000000000080819E
:3D2438000000000000000000000000000000000000000000000000000000000000000000000000000000000000000000000000000000000006000000000000808160
:3D2475000000000000000000000000000000000000000000000000000000000000000000000000000000000000000000000000000000000006000000000000808123
:3D24B200020000000000000000000000000000000000000000000000000200000000000000000000000000000000000000000000000000000000000000048008C39A
:3D24EF000200000000000000000000000000000000000000000000006000000000000000000000000000000000000000000000000000000000000000988001888D20
:3D252C00020000000000000000000000000000000000000000000000000000000000000000000000000000000000000000000000000000000000000000000008ED7B
:3D256900020000000000000000000000000000000000000000000000400000000000000000000000000000000000000000000000000000000000000010000108AD2D
:3D25A600000000000000000000000000000000000000000000000000800100000000000000000000000000000000000000000000000000000000000060000600FE13
:3D25E3000E0000000000000000000000000000000000000000000000800100000000000000000000000000000000000000000000000000000000000060000600F0D6
:3D2620001E0000000000000000000000000000000000000000000000800100000000000000000000000000000000000000000000000000000000000060000688E808
:3D265D00000000000000000000000000000000000000000000000000800100000000000000000000000000000000000000000000000000000000000060000600FE5B
:3D269A00000110000110000110000110000110000110000110000110000110000000000040000440000440000440000440000440000440000440000440000480E79F
:3D26D700000000000000000000000000000000000000000000000000000000000000000000000000000000000000000000000000000000000000000000000080E75F
:3D271400800118800118800118800118800118800118800118800118800118000000000060000660000660000660000660000660000660000660000660000680E72A
:3D275100800008800008800008800008800008800008800008800008800008000000000020000220000220000220000220000220000220000220000220000280E7EA
:3D278E00000000000000000000000000000000000000000000000000100000000000000000000000000000000000000000000000000000000800002000000000F5E1
:3D27CB00000000000000000000000000000000000000000000000000000000000000000000000000000000000000000000000000000000000000000000000080E76A
:3D280800000000000000000000000000000000000000000000000000000000000000000000000000000000000000000000000000000000000000000000000080E72C
:3D284500000000000000000000000000000000000000000000000000800000000000000000000000000000000000000000000000000000000000000020000200EFC5
:3D288200000000000000000000000000000000000000000000000000100000000000000000000000000000000000000000000000000000000800002000000000F5EC
:3D28BF00000000000000000000000000000000000000000000000000000000000000000000000000000000000000000000000000000000000000000000000080E775
:3D28FC000000000000000000000000000000000000000000000000000000000000000000000000000000000000000000000000000000000000000000000000F0901F
:3D293900000000000000000000000000000000000000000000002000000000000000000000000000000000000000000000000000000000000000000000000080E5DC
:3D297600000000000000000000000000000000000000000000000000000000000000000000000000000000000000000000000000000000000000000022000800E515
:3D29B300000000000000000000000000000000000000000010000000400000000000000000000000000000000000000000000000000000000000100000000080A661
:3D29F0000000000000000000000000000000000000000000000000000000001000000000000000000000000000000000000000000000000080000000000000B0CC9E
:3D2A2D00000000000000000000000000000000000000000000000000000000000000000000000000000000000000000000000000000000000000000000000080E705
:3D2A6A00000000000000000000000000000000000000000000000000000000000000000000000000000000000000000000000000000000000000000000000080E7C8
:3D2AA700000000000000000000000000000000000000000000000000000000000000000000000000000000000000000000000000000000000000000000000080E78B
:3D2AE400000000000000000000000000000000000000000000000000000000000000000000000000000000000000000000000000000000000000000000000080E74E
:3D2B2100000000000000000000000000000000000000000000000000000000000000000000000000000000000000000000000000000000000000000000000080E710
:3D2B5E000000000000000000000000000000000000000000000000000000000000000000000000000000000000000000000000000000000000000000000000C0A3D7
:3D2B9B00000000000000000000000000000000000000000000000000000000000000000000000000000000000000000000000000000000000000000000000080E796
:3D2BD800000000000000000000000000000000000000000000000000000000000000000000000000000000000000000000000000000000000000000000000080E759
:3D2C1500000000000000000000000000000000000000000000000000000000000000000000000000000000000000000000000000000000000000000000000080E71B
:3D2C5200000000000000000000000000000000000000000000000000000000000000000000000000000000000000000000000000000000000000000000000080E7DE
:3D2C8F00000000000000000000000000000000000000000000000000000000000000000000000000000000000000000000000000000000000000000000000080E7A1
:3D2CCC00000000000000000000000000000000000000000000000000000000000000000000000000000000000000000000000000000000000000000000000080E764
:3D2D0900000000000000000000000000000000000000000000000000000000000000000000000000000000000000000000000000000000000000000000000080E726
:3D2D4600000000000000000000000000000000000000000000000000000000000000000000000000000000000000000000000000000000000000000000000080E7E9
:3D2D8300000000000000000000000000000000000000000000000000000000000000000000000000000000000000000000000000000000000000000000000080E7AC
:3D2DC000000000000000000000000000000000000000000000000000000000000000000000000000000000000000000000000000000000000000000000000080E76F
:3D2DFD00000010000100000000800812000100800810000100000010000140000000000000000040000040001020020400000000000040000000000440000480E65F
:3D2E3A00000008800000000000002008800000002008800000000008800008000000000000000020000020000200080200000000000020000000000220000200E77C
:3D2E7700000000000000000000000000000000000000000000000000000000000000000000000000000000000000000000000000000000000000000000000080E7B7
:3D2EB400000000000000000000000000000000000000000000000000000000000000000000000000000000000000000000000000000000000000000000000080E77A
:3D2EF10040100EE1100441100441380EE1100441380EE1100441100EE1100E0100000000100441380441388443108E4310044110044138044110844338844300C531
:3D2F2E00601896611986611886615896611986615896611986611896611996010000000018866158866158866518966518866118866158866118866558866580E61E
:022F6B00FFFF66
:00000001FF
